:1064590000FFFF02FFFF0301FA0400FA0500030A27
:10646900FFFF0BFFFF0CFFFF0D00000E00040F01E3
:106479006410009612FFFF13FFFF14010217010AAF
:106489001801FA1905321A010A1B01FA1C05321FF3
:10649900FFFF20FFFF23FFFF24FFFF2A00FA2B0045
:1064A900FA2C50782DFFFF2EFFFF30FFFF32507876
:1064B9003300003432FA35FFFF36FFFF37FFFF386C
:1064C900FFFF3A00003CFFFF3EFFFF3F000140FF96
:1064D900FF411450420A5A430AC844FFFF4500B419
:1064E90046FFFF4CFFFF50040451059652FFFF532E
:1064F9000B4654FFFF57FFFF5AFFFF5BFFFF5CFF8F
:10650900FF5EFFFF5FFFFF64021C67FFFF6AFFFF7B
:106519006B00006C329673000074000078013279C8
:1065290001327E006481006484FFFF8A00019D0AB4
:10653900969E00019FFFFFA0013CA2000AA3FFFF56
:10654900A4FFFFA5FFFFA6FFFFA7FFFFA8FFFFA965
:10655900FFFF0100001500022FFFFF47013C480221
:10656900035600004EFFFF58000061FFFF66FFFF62
:1065790085FFFF86FFFF87FFFF890000990000A1C3
:10658900FFFFFAFAFA0065006F00790083008D00B9
:106599009700A100AC00B600C000CA00D400DE001C
:1065A900E800F20058006000680070007800800080
:1065B900880090009800A000A800B000B800C100B1
:1065C900C800D000D800DF00E600EE00F600410068
:1065D90047004D00530059005F0065006C007100D1
:1065E90077007D00830089008F0095009B00A20041
:1065F900A700AC00B200B900C000C500CA00D200B3
:09660900D500DD00E100E700EF1F
:10331000900885E0900111F0900886E0900080F020
:10332000900887E09000A0F0900888E09000C9F035
:10333000900889E0900075F090088AE09000BBF05A
:1033400090088BE09000D9F090088CE09000ADF0F0
:1033500090088DE09000CBF090088EE09000FBF09C
:1033600090088FE090015FF0900890E0900160F08D
:10337000900891E0900161F090015FE0700C900185
:1033800060E07006900161E060028004C22080026B
:10339000D220743690014AF0743090014BF0742DB5
:1033A00090014CF0743290014DF0742090014EF079
:1033B000743490014FF07443900150F0747990018F
:1033C00051F0746C900152F07420900153F07446E7
:1033D000900154F07475900155F07465900156F0A9
:1033E000746C900157F07420900158F02290087D81
:1033F000E0FEA3E0FF7402D39F74019E400C906432
:1034000059120048E493F599801290087DE0FEA3DC
:10341000E0FF906459120048E493F59990087D12FA
:10342000673290087DE0FEA3E0FFEFB43507EEB40D
:103430000103754D002285F97385FA747E017F00C2
:10344000E574126724E5732FFF50010E8E5A8F5BCF
:10345000900015E0FCA3E0FDEF2DFDEE3CFC8C5C44
:103460008D5D2275A71085F97385FA747E017F0042
:10347000E574126724E5732FFF50010E8E5A8F5B9F
:103480009000D9E0B40210AC2CAD2DEF2DFDEE3C38
:10349000FC8C5C8D5D8016AE5AAF5B900015E0FC35
:1034A000A3E0FDEF2DFDEE3CFC8C5C8D5D22AE5A61
:1034B000AF5B74068E048F05FF1267148C5C8D5D04
:1034C000AE5AAF5B74068E048F05FF12673F8C5AAD
:1034D0008D5BC200E55B455A60137406C3955BFFC4
:1034E000E4955AFE8E5A8F5B785C126777E573A875
:1034F0005CB80015D3955D4010E573C3955DFFE49E
:10350000955CFE8E5C8F5D8012E573243CC3955DF7
:10351000FFE4955CFE8E5C8F5DD200AE5CAF5D74A7
:103520003B6F4E6006743C6F4E701AAE5CAF5D74BC
:103530003B6F4E70057573018003757302755D3ABC
:10354000755C00800375730022900087E0B401046D
:10355000C2078002D207900088E0B40104C208804C
:1035600002D2089000C5E075F0E1A4FFAEF0740A45
:103570008E048F05FF126714900875ECF0A3EDF030
:1035800074078C068D0712672474038E048F05FF61
:10359000126714900011ECF0A3EDF07E017F009013
:1035A0000083E01267249000C6E08E048F05FF12AE
:1035B0006714740AFF1267148D609000CFE075F0F5
:1035C000E1A4FFAEF0740A8E048F05FF1267149019
:1035D0000879ECF0A3EDF09000D1E060139000D1F9
:1035E000E0F5F0741684FF7E00EF9008A1F08006ED
:1035F00074649008A1F09000C7E0900062F0900120
:1036000013E090006DF0900115E0FE9000C3E08E95
:103610000088F0A4FFAEF0EF9008A9F0900111E04F
:10362000900885F09000A0E0900887F0900075E089
:10363000900889F09000FBE090088EF090015FE028
:1036400090088FF0900160E0900890F0900161E0A8
:10365000900891F0A220B3401690015FE0700C90AA
:103660000160E07006900161E060028002C220907B
:10367000015FE0B4300F900160E0B4470890016151
:10368000E0643B60028004D2218002C22174E39096
:103690000061F09000B0E0B40B0874E3900061F0BA
:1036A000805A9000B0E0B419129000C6E09065799D
:1036B00012008CE493900061F080419000B0E0B47F
:1036C0001E129000C6E090659712008CE493900063
:1036D00061F080289000B0E0B428129000C6E0901D
:1036E00065C112008CE493900061F0800F9000B0EF
:1036F000E0B446089000A7E0900061F0900088E0F8
:1037000070089000C9E064046002800874039000AF
:10371000C9F0D21F900065E0FE9000ADE0B50657FD
:10372000900067E0FE9000CBE0B5064B900066E0AD
:10373000FE9000D9E0B5063F90006AE0FE90008060
:10374000E0B50633900068E0FE9000BBE0B50627C8
:10375000900069E0FE9000C9E0B5061B90006BE0A8
:10376000FE9000E6E0B5060F90006CE0FE9000E7EA
:10377000E06E7003023935900080E0B401067400F9
:10378000900080F0900080E0B4020674009000CBBE
:10379000F0900080E0B4030674009000D8F0900030
:1037A000CBE0D394014027741B9000FEF07400908E
:1037B00006C9F074009006CAF07400900095F0906D
:1037C00000ADE0B4020674019000ADF080339000CB
:1037D000ADE0B4021A74009000FEF074009006C9C7
:1037E000F074009006CAF0741B900095F08012747B
:1037F000009000FEF0741B9006C9F07400900095D4
:10380000F09000ADE06014741C900094F07400908F
:1038100006CDF074009006CEF0800C7400900094F9
:10382000F0741C9006CDF09000E6E06014741990DE
:103830000100F074009006C1F074009006C2F080A0
:103840000C7400900100F074199006C1F09000E72C
:10385000E06014741A900101F074009006C5F074D1
:10386000009006C6F0800C7400900101F0741A906C
:1038700006C5F09000D9E0701A74059006D1F07476
:10388000069006D5F074079006D9F074089006DD0E
:10389000F0803074009006D1F074009006D2F0747D
:1038A000009006D5F074009006D6F074009006D90A
:1038B000F074009006DAF074009006DDF074009069
:1038C00006DEF0D21F9000ADE0900065F09000D9C8
:1038D000E0900066F09000CBE0900067F09000BBB5
:1038E000E0900068F09000C9E0900069F0900080DE
:1038F000E090006AF09000E6E090006BF09000E746
:10390000E090006CF0900080E0900886F09000C994
:10391000E0900888F09000BBE090088AF09000D911
:10392000E090088BF09000ADE090088CF09000CB18
:10393000E090088DF09000E3E0B40117900021744E
:103940000FF0A374FFF0900023E4F0A3F074029052
:1039500000E3F09000E3E0B40341900023E0FEA315
:10396000E0FF900021E0FCA3E0FD12676F741012ED
:1039700067247408120039EF90005EF0EF7006744F
:10398000FF90005EF074009000E3F0900022E09061
:10399000005FF0900021E0900060F0900074E090F3
:1039A0000071F0900073E0900070F09000A2E0C30E
:1039B000941E50569000A2E0F404241E900072F071
:1039C000900072E075F00684FF7E008F73900072A5
:1039D000E075F00684ADF07C008D74900070E0D34B
:1039E0009574400D900070E0C39574900070F08065
:1039F0000F900070E02406C39574900070F005737A
:103A0000900071E02573900071F0900071E09000DB
:103A10003DF090003DE0241E90003EF090003DE01F
:103A2000D39478400B90003DE0C3947890003DF033
:103A300090003EE0D39478400B90003EE0C3947831
:103A400090003EF0C22390003DE0D3943C400D90A6
:103A5000003DE0C3943C90003DF0D223C22490008E
:103A60003EE0D3943C400D90003EE0C3943C900077
:103A70003EF0D224900041E4F090003DE0643B60D1
:103A80000790003DE0B43C2090003DE0B43B06745C
:103A900002900041F090003DE0B43C06900041747B
:103AA00001F090003D7401F0900042E4F090003E7F
:103AB000E0643B600790003EE0B43C2090003EE0B4
:103AC000B43B067402900042F090003EE0B43C0625
:103AD0009000427401F090003E7401F0900074E098
:103AE000FE9000D7E02E900044F0900044E0D39484
:103AF0003C400B900044E0C3943C900044F09000A4
:103B000044E0D3943C400B900044E0C3943C9000CC
:103B100044F0900044E0641E6007900044E0B43C30
:103B200006900044E004F0900044E0641D600790BB
:103B30000044E0B43B06900044E014F0900044E000
:103B4000D3943C400B900044E0C3943C900044F07C
:103B5000900044E0D3941E400D900044E0C3941EB6
:103B6000900045F0800A900044E0241E900045F04B
:103B700075511E9000BAE090003FF090003FE07554
:103B8000F01E84AFF07E00EF4E700690003FE00420
:103B9000F090003FE00475F01E84AFF07E00EF4E21
:103BA000700690003FE014F090003FE0B47906907A
:103BB000003F7401F090003FE0D3943C400F900030
:103BC0003FE0C3943C90003FF0D21A8002C21A90AA
:103BD000003FE0D3941E400D90003FE0C3941E9040
:103BE0000040F0800A90003FE0241E900040F02248
:103BF000C293C294C291C292C287C290E5B554EFFB
:103C0000F5B5E5B554DFF5B5C296C295C2A0C29729
:103C1000C2A2C2A1E5B554BFF5B5E5B5547FF5B56F
:103C2000E5B554FBF5B5C209755E469000BDE07080
:103C300005756D028003756D037555007554009010
:103C4000000874FFF0A374DCF0C20EC21174C890B7
:103C50000035F074C8900039F0755300755200C2F9
:103C600004754600E56FB40903756F007563009035
:103C70000017E4F0A3F0757010C20CC20DC20375FA
:103C8000570075560090000AE4F0A3F090000CE491
:103C9000F0A3F0C22875590075580090007FE075B8
:103CA000F032A4FFAEF090001FEEF0A3EFF0900012
:103CB0006EE4F090006FE4F0C222D217C216D21860
:103CC000C219C21AC21B22755B00755A00AE5AAFE8
:103CD0005B7402C39F74019E5003023D859064593A
:103CE000120048E4939000731267550FBF00010E55
:103CF000E0FC906459120048ECFEE493FFEEC39F91
:103D00005026AE5AAF5B0FBF00010E9064591200EF
:103D100048AE5AAF5BE493FC906459120048E493B8
:103D2000900073126755ECF0AE5AAF5B9064591275
:103D30000048E493900073126755E0FC90645B12B6
:103D40000048ECFCE493FDECD39D401990645B12B9
:103D50000048E493FC906459120048E49390007387
:103D6000126755ECF0AE5AAF5B74022FFF50010E94
:103D70008E5A8F5B785B740126F6500418E436F691
:103D80004003023CCD22755B00755A00AE5AAF5B12
:103D90007433BE00039F5003023E5390655B1200D4
:103DA00048E4939000731267550FBF00010EE0FCCA
:103DB00090655B120048ECFEE493FFEEC39F502633
:103DC000AE5AAF5B0FBF00010E90655B120048AEAC
:103DD0005AAF5BE493FC90655B120048E49390005B
:103DE00073126755ECF0AE5AAF5B90655B120048FA
:103DF000E493900073126755E0FC90655D120048F3
:103E0000ECFCE493FDECD39D401990655D120048F5
:103E1000E493FC90655B120048E493900073126792
:103E200055ECF0AE5AAF5B742D6F4E7006755B3378
:103E3000755A00AE5AAF5B74022FFF50010E8E5AB6
:103E40008F5B785B740126F6500418E436F6400365
:103E5000023D8C22E50C905FF8F8282873023F1A87
:103E600075E700A231B34008E5B54408F5B5800612
:103E7000E5B554F7F5B575E710023F1A75E700A2EE
:103E800031B34008E5B54402F5B58006E5B554FD0B
:103E9000F5B575E710023F1AA23192A2807CA231DB
:103EA00092A1807675E700A231B34008E5B54440A1
:103EB000F5B58006E5B554BFF5B575E710805B75BF
:103EC000E700A231B34008E5B54480F5B58006E5CA
:103ED000B5547FF5B575E7108040A2319287803ADE
:103EE000A2319290803475E700A231B34008E5B565
:103EF0004410F5B58006E5B554EFF5B575E71080CB
:103F00001975E700A231B34008E5B54420F5B58046
:0A3F100006E5B554DFF5B575E710BE
:105FF800023E5D023E60023E7C023E98023E9E02E8
:106008003EA4023EBF023EDA023EE0023EE6023F06
:016018000186
:103F1A002285F97385FA747E017F00E5741267249D
:103F2A00E5732FFF50010E8E5A8F5BAC5CAD5DEFCF
:103F3A002DFDEE3CFC8C5C8D5DD293D294D291D255
:103F4A0092E55DF5FBE55CF5FCE55DF5E9E55CF51B
:103F5A00EAE55DF5EBE55CF5ECE55DF5EDE55CF5CF
:103F6A00EE2275A71085F97385FA747E017F00E544
:103F7A0074126724E5732FFF50010E8E5A8F5B7EF1
:103F8A00017F769000F8E0126724AC5AAD5BED2F02
:103F9A00FFEC3EFE8E5C8F5DE55DF5FDE55CF5FEB2
:103FAA00900062E4F075A7007412900047F0228531
:103FBA00F97385FA747E017F00E574126724E5734C
:103FCA002FFF50010E8E5A8F5B900011E0FCA3E088
:103FDA00FDEF2DFDEE3CFC8C5C8D5DE55DF5FDE5B0
:103FEA005CF5FE220564229000BBE0B40353900006
:103FFA00D9E0B4012EA2D8B34004C293C287A2D991
:10400A00B34004C294C290A2DAB34008C291E5B5A3
:10401A0054EFF5B5A2DBB34008C292E5B554DFF51B
:10402A00B5801CA2D8B34002C293A2D9B34002C23F
:10403A0094A2DAB34002C291A2DBB34002C29280D8
:10404A002EA2D8B34012C293C2919000D9E0600860
:10405A00C287E5B554EFF5B5A2D9B34012C294C2EE
:10406A00929000D9E06008C290E5B554DFF5B5A298
:10407A00DCB34030A29650067419900047F0A2951E
:10408A0050067419900047F0A2A0500674199000C7
:10409A0047F0A29750067419900047F0C296C2954D
:1040AA00C2A0C29775D8402285A77275A710A2D858
:1040BA00B34002C287A2D9B34002C290A2DAB34087
:1040CA0006E5B554EFF5B5A2DBB34006E5B554DF16
:1040DA00F5B5A2DCB340089000C7E0900062F07525
:1040EA00D8408572A72290F800E4936406600280A3
:1040FA00FE75B50075840175A70075FFA075EF06FA
:10410A00900043E4F075C91075A70F75A1C775A78C
:10411A000075D90075CE0C75A70F75F1FE75F2FF03
:10412A0075F30775F47875A4BA75A5FF75A60775B2
:10413A00AE0075AFFF75D48175D5FF75D6FF75D7FB
:10414A00FF75A70075A20175A14775F80975D80012
:10415A0075D90475DA0975DB0975DC0975DD097528
:10416A00DE0975D84075A71075D80075D90475DAB7
:10417A000975DB0975DC0975DD0975DE0975D84035
:10418A0075A70075E60875E71075BC0175BE04755C
:10419A00BD6C75BE0775BDA075BE0875BD0175BC41
:1041AA000075BB1875BC2075BA0875E88075D113FF
:1041BA0075A70F75E10575E20075C740123BF075EA
:1041CA009700759780740A1267047597C0E597542B
:1041DA0020700280F8758F0275A700D2AF7598001B
:1041EA0075A90C75A70F75AB4375ADFB75AC1E753C
:1041FA00A71075C91875CA0075CB0075C80475A7CC
:10420A0000758912758E04758C00758A00C2A9D250
:10421A008C758D00758B00D2ABD28E75B62075D990
:10422A0044C299C22774C8F5097508001200F875C6
:10423A00A70FE5FB900051F0E5FA900052F0E5F97E
:10424A00900053F075A70090F800E493F527120246
:10425A0017900886E0D394035007900886E0B401CB
:10426A00067400900886F074019000BCF0900886ED
:10427A00E0906019F8282873802A802875A70F759E
:10428A00F30F75A700A2A3400674029000BCF08049
:10429A001375A70F75F31775A700A2A44006740239
:0442AA009000BCF0D4
:0C60190002428202428402428602429B44
:1042AE009000BCE0B4022AC2251205B6740290003A
:1042BE00BCF0900886E0906025F828287380108066
:0F42CE000E74009000CBF0800674009000D8F0C2
:0C6025000242CB0242CD0242CF0242D721
:1042DD008028D2251204D574019000BCF090088678
:1042ED00E0906031F82828738010800E74009000E3
:0A42FD00CBF0800674009000D8F0AA
:0C6031000242F50242F70242F90243016C
:104307001233109000C6E07006740A9000C6F09051
:1043170000A7E0700674E39000A7F09000ADE004FA
:10432700900065F0123CC7123D8612354990F80798
:10433700E493900058F0900058E0440A900058F039
:10434700900058E054FE900058F07406900049F031
:10435700740190004AF090F802E49390004BF074D7
:104367000390004CF0740590004DF0747090004E6F
:10437700F0740390004FF07406900050F090F8042A
:10438700E493900054F07400900055F090F805E421
:1043970093900056F090F806E493900057F074FF5E
:1043A700900059F09000E2E090005EF0900099E0F4
:1043B70090005FF090009AE0900060F0A2B6B39290
:1043C70005A2B3B39206A2A4B3921DA2A3B3921EF1
:1043D70090005AE4F0756F00743A900773F074FD1B
:1043E700900774F090005BE4F0756E01900047E46D
:1043F700F09000BDE0B40106741A900047F0C21CAB
:10440700756300C20AD20BC203757100C21FC226B0
:1044170012009E755F00756B0075610075653275DA
:104427006600756700756800756900756A00900019
:1044370017E4F0A3F0756C00D2B2D2A4D2B0D2B117
:10444700D2A3D2A7D2A6D2A5D2B790007FE0D394A9
:10445700FA400674FA90007FF07E017F00900060BA
:10446700E012672490005FE02FFF50010E900021BB
:10447700EEF0A3EFF0EFD394FFEE940F4007900018
:1044870021E4F0A3F090005EE0700674FF90005EF8
:10449700F09000BDE07005756D028003756D0390A7
:1044A70000BEE0D39401400674009000BEF0900077
:1044B700C4E0C3940A5006740A9000C4F09000CE7A
:1044C700E0700674019000CEF09000CEE0B4FF06D5
:1044D70074FE9000CEF09000D5E0D394FE400674B1
:1044E700FE9000D5F09000FBE0D3940240067401E3
:1044F7009000FBF0900111E0D39401400674019005
:104507000111F074019000DBF074019000DCF0748D
:10451700009000E3F074009000FFF0740090010336
:10452700F074009006B9F074009006BDF0D29C902C
:1045370000AEE0D39404400674049000AEF09000FF
:10454700E0E0D39404400674049000E0F0E570D3F3
:10455700941040037570109006BAE0D3940C40068F
:1045670074009006BAF09006BEE0D3940C4006742F
:10457700009006BEF09006C2E0D3940C400674008B
:104587009006C2F09006C6E0D3940C4006740090E3
:1045970006C6F09006CAE0D3940C40067400900655
:1045A700CAF09006CEE0D3940C400674009006CE75
:1045B700F09006D2E0D3940C400674009006D2F037
:1045C7009006D6E0D3940C400674009006D6F0907F
:1045D70006DAE0D3940C400674009006DAF09006F1
:1045E700DEE0D3940C400674009006DEF0D2EC7542
:1045F700CF01A298B34005C298120697E54D600611
:10460700A299B3B340028005C299120B78E54E64B4
:10461700016005E54EB4040280D5C28E7E107F008E
:10462700E564126724E58D75F010A4FDACF0EF2D5D
:10463700FDEE3CFCE58B75F01084FF7E00ED2FFF4F
:10464700EC3EFE8E548F55D28E9000A0E06009900C
:1046570000A0E0C3943D4002805C900019126732CD
:10466700900019E0FEA3E0FF90001BE0FCA3E0FD33
:10467700EFB50542EEB5043EB214A204B340197576
:10468700E700A214B34008E5B54404F5B58006E594
:10469700B554FBF5B575E71090001BE0FEA3E0FFEE
:1046A70090001DE0FCA3E0FDEF2DFDEE3CFC90002B
:1046B7001BECF0A3EDF09000ADE060099000ADE0D9
:1046C700C394034003024770122745A204B350095D
:1046D70090005AE0C3942D40028006900097E0F5C1
:1046E70045E54575F002A4FFAEF090087BEEF0A318
:1046F700EFF0900084E0C395614007E55FC39560E4
:10470700500790087BE4F0A3F075E700AE2EAF2FBB
:1047170090087BE0FCA3E0FDEFD39DEE9C4020E5F5
:10472700B5547FF5B59000ADE0B402099000CBE039
:10473700C3940240028006E5B54440F5B580279052
:10474700005AE0C39444501EE5B54480F5B5900087
:10475700ADE0B402099000CBE0C3940240028006AA
:10476700E5B554BFF5B575E7109000ADE0B4032A81
:1047770012286075E700AE2EAF2F90087BE0FCA3F0
:10478700E0FDEFD39DEE9C4008E5B54480F5B5808C
:1047970006E5B5547FF5B575E710900088E0600928
:1047A700A2B3300601B3B340028056A2B33006016C
:1047B700B3404EA2B3300801B34039A2174030903E
:1047C700006DE0D3955E402590006FE07013900078
:1047D7006EE0B4010690006F7401F090006EE00483
:1047E700F0A216B3400590006EE4F0D216D217A2DD
:1047F70008B39206A208B330B301B34004A20892EB
:1048070006A2B6300501B35003024ED0A2B630055A
:1048170001B35003024ED0A2B6300701B3500302D2
:104827004D7C756E009000A0E0B43D1975E700A2BD
:1048370007B34008E5B554FBF5B58006E5B5440474
:10484700F5B575E710055EA209B3B35013AE54AFC3
:1048570055900008E0FCA3E0FDEDC39FEC9E4003EC
:10486700024A4BE56DB4032EA228B34022E55EB49D
:104877003B03756D01E55EC3943B5006900047749A
:1048870001F0E55ED3943B40067402900047F07553
:104897005E01D2288062E56DB4020A756D01755E0E
:1048A7003BC216C218E55EB43B05755E01804990B0
:1048B7000047E07034E55EC3943B500690004774B0
:1048C70001F0E55ED3943B40067402900047F0E5A3
:1048D7005EC3943B5002D21CE55ED3943B4002D2A8
:1048E7001CC296C295C2A0C2979000BDE0B4010554
:1048F700123BF08003755E01AE56AF57AC54AD5511
:10490700EF2DFDEE3CFC74028C068D071200398EEC
:10491700568F579000A0E060099000A0E0C3943D37
:1049270040028049900019E0FEA3E0FF9000A0E05C
:104937008E048F05FF12671474018C068D07120011
:104947003990001DEEF0A3EFF090001DE0F8A3E012
:1049570090001BC8F0A3C8F0900019E4F0A3F0C2C0
:104967001475E700E5B554FBF5B575E710A2A4B3D8
:104977004002C21DA2A3B34002C21EA21CB3400242
:10498700C21C75E700B226A2264008E5B554FBF520
:10499700B58006E5B54404F5B575E710B219900082
:1049A7006FE0B40111A216B34004D2198002C219F4
:1049B700740290006FF090006FE0C394025006A25B
:1049C70004B3B340028006740290006FF09000C9F0
:1049D700E0640460079000BBE0B40362900088E0E5
:1049E700600690006FE07002800DA218301601B3C8
:1049F700400590006EE4F09000BDE064016006A2FF
:104A070022B3B35017900088E06009A2163018014E
:104A1700B3B3400280067405900047F0B218A2179E
:104A2700B3401BA216B34004D2188002C2189000EC
:104A3700BDE0700690006FE070028002D222C216BD
:104A4700C217803AAE56AF57AC54AD55EF2DFDEEB9
:104A57003CFC74018C068D071200398E568F57E582
:104A67006DC39402500DAC54AD5574B8C39D740B0F
:104A77009C40028009123BF07406900047F0E55E07
:104A8700B43B127403900047F0D21C9000BDE0B411
:104A97000103123BF0AE58AF59AC54AD55EF2DFDA5
:104AA700EE3CFC8C588D59AE54AF55EFD39DEE9C20
:104AB700401190000FE0FAA3E0FBEBC394E8EA94FF
:104AC700034002800690000F12673290000CE0FE50
:104AD700A3E0FFAC54AD55EF2DFDEE3CFC90000C70
:104AE700ECF0A3EDF09000BDE0B40118AE54AF5563
:104AF70074051267247401120039900008EEF0A3C0
:104B0700EFF08011AE54AF5574021267249000087D
:104B1700EEF0A3EFF0C28E758D00758B0075640003
:104B2700755501755400D28EE55E240E75F00F841D
:104B3700AFF07E00EF4E6003024BC4E56D6013AE2D
:104B470056AF57740F12672490000AEEF0A3EFF0E8
:104B5700800F90000CE0F8A3E090000AC8F0A3C80B
:104B6700F090000AE0FEA3E0FFEF4E600B7C777D3C
:104B7700DF1266128E528F5390000CE4F0A3F0AE52
:104B870052AF537428BE00039F5010E5632FFF50A8
:104B9700010E74011200398E528F538553639000B2
:104BA700C4E0A852B8000DD395534008E5539000D0
:104BB70046F080099000C4E014900046F09000BBD6
:104BC700E0B4030890003FE0655E6002800EA21922
:104BD700301A01B34004D21B8002C21BE55E640B8E
:104BE7006005E55EB429099000ADE0600312241169
:104BF700900044E0655E6007900045E0B55E037590
:104C07006F00A20AB35006A209B3B34003024CBC1B
:104C1700900079E0B401739000FBE0B40214120D28
:104C270019900063E075F0BEA4FFAEF08E5C8F5D57
:104C37008056E56775F00A84FF7E009005731200C1
:104C470048E0F55B755A00AE5AAF5B90009EE012E4
:104C5700672474648E048F05FF1267148C5C8D5D66
:104C6700E55D90000EF0AE5AAF5B900077E01267FB
:104C77002474648E048F05FF12671474BE8C068D2E
:104C8700071267248E5C8F5D8017900077E075F0C0
:104C9700BEA4FFAEF08E5C8F5D90009EE090000E8C
:104CA700F0E561C394CC5006E55D455C7002800376
:104CB700123F1BD20AE56DB40106E55E641160027E
:104CC70080189000C9E0B4040575700380097570F9
:104CD700019000487401F0756D00E56D6003024DA9
:104CE700779000C0E0600D900062E0A852B800061F
:104CF7009553400280389000C0E0B4021790003D01
:104D0700E0655E600790003EE0B55E037570037571
:104D17006C00800CC201756C00900017E4F0A3F0E2
:104D2700900062E060067409900047F080429000AE
:104D37003DE0655E600790003EE0B55E339000C9D8
:104D4700E0B4040FA222B3400575700180037570AB
:104D570003800375700190003DE0B55E0690004842
:104D67007401F090003EE0B55E067402900048F0D2
:104D7700A207B39205A207B330B601B35003024EA0
:104D8700D0756E019000A0E0B43D1975E700A20749
:104D9700B34008E5B54404F5B58006E5B554FBF521
:104DA700B575E710A227400575FFA0D22775E70064
:104DB700E5B54401F5B575E710742D90005AF0A2DA
:104DC700079205E55ED3944A4014D209E55ED39471
:104DD70085400B7404900047F0D21C755E46900026
:104DE700C8E0B40107E56AC3941440028009123B86
:104DF700F07413900047F0E56AC394415009740EAC
:104E0700900047F0123BF090004FE0FE90004BE01F
:104E1700C39E400990004BE0D39408400974FB906F
:104E27000047F0123BF0900054E06015900054E00A
:104E3700FE90004EE06E600974FE900047F0123B52
:104E4700F0900886E060069000F8E06002807A74CF
:104E5700019000BCF0900886E090603DF828287328
:104E670080188016A2A3400674029000BCF0800A46
:0A4E7700A2A4400674029000BCF0F3
:0C603D00024E67024E69024E6B024E7765
:104E81009000BCE0B40105A225B340028019D225EF
:104E9100123BF01204D574019000BCF0123310D211
:104EA1001F741B900047F09000BCE0B40206A225DD
:104EB100B3B340028019C225123BF01205B6740249
:104EC1009000BCF0123310D21F741B900047F0A267
:104ED1001CB34008C296C295C2A0C2979000F8E0E8
:104EE100600CAE52AF537414BE00059F4002803770
:104EF100900080E0906049F8282873802A8028A2D9
:104F0100A3B35005A21EB340028005123F6CD21E0E
:104F11008015A2A4B35005A21DB340028005123F23
:074F21006CD21D800280002C
:10604900024EFC024EFE024F00024F13024F26027F
:026059004F28CE
:104F2800A20CB3B3500890003FE0655E60030251E5
:104F380061A202B35006A201B3B3400302515D90CF
:104F480000BBE0B40302800302511C90006FE0B480
:104F580002028003025103A21BB350030250301215
:104F6800343690010CE0601F900015E0FEA3E0FFCE
:104F7800900104E012672474C88E048F05FF12673D
:104F8800148C5C8D5D800A900015E0F55CA3E0F55B
:104F98005DAE5CAF5D745E12672474058E048F0588
:104FA800FF126714AE5AAF5BED2FFFEC3EFE8E5C2E
:104FB8008F5DE55DF5FBE55CF5FCD293A203B3409C
:104FC80002D2879000D9E0B4025B12346390010CDE
:104FD800E0D39404401BAE2CAF2D900108E012677B
:104FE8002474C88E048F05FF1267148C5C8D5D8055
:104FF80006852C5C852D5DAE5CAF5D745E12672402
:1050080074058E048F05FF126714AE5AAF5BED2F3F
:10501800FFEC3EFE8E5C8F5DE55DF5FBE55CF5FC27
:1050280075A700D28702510112343690010CE0D3E3
:105038009403401F900015E0FEA3E0FF900106E0F6
:1050480012672474C88E048F05FF1267148C5C8D58
:105058005D800A900015E0F55CA3E0F55DAE5CAFFD
:105068005D745E12672474058E048F05FF12671441
:10507800AE5AAF5BED2FFFEC3EFE8E5C8F5DE55DBB
:10508800F5EBE55CF5ECD291A203B34006E5B54437
:1050980010F5B59000D9E0B4025F12346390010CAA
:1050A800E0D39406401BAE2CAF2D90010AE01267A6
:1050B8002474C88E048F05FF1267148C5C8D5D8084
:1050C80006852C5C852D5DAE5CAF5D745E12672431
:1050D80074058E048F05FF126714AE5AAF5BED2F6F
:1050E800FFEC3EFE8E5C8F5DE55DF5EBE55CF5EC77
:1050F80075A700E5B54410F5B58017123436E55D9F
:10510800F5FBE55CF5FCE55DF5EBE55CF5ECD293CC
:10511800D2918041123436E55DF5FBE55CF5FCD2B1
:1051280093D291A203B34008D287E5B54410F5B5F0
:105138009000D9E0B4021E123463E55DF5FBE55C2E
:10514800F5FCE55DF5EBE55CF5EC75A700D287E5C8
:10515800B54410F5B5C20CD20DA20DB3B3500890EA
:105168000040E0655E600302539DA202B35006A2B0
:1051780001B3B340030253999000BBE0B40302802B
:105188000302535890006FE0B40202800302533FB9
:10519800A21BB3500302526C12343690010CE0D3B8
:1051A8009401401F900015E0FEA3E0FF900105E088
:1051B80012672474C88E048F05FF1267148C5C8DE7
:1051C8005D800A900015E0F55CA3E0F55DAE5CAF8C
:1051D8005D745E12672474058E048F05FF126714D0
:1051E800AE5AAF5BED2FFFEC3EFE8E5C8F5DE55D4A
:1051F800F5E9E55CF5EAD294A203B34002D29090B7
:1052080000D9E0B4025B12346390010CE0D394053A
:10521800401BAE2CAF2D900109E012672474C88E94
:10522800048F05FF1267148C5C8D5D8006852C5CED
:10523800852D5DAE5CAF5D745E12672474058E04C7
:105248008F05FF126714AE5AAF5BED2FFFEC3EFEE1
:105258008E5C8F5DE55DF5E9E55CF5EA75A700D242
:105268009002533D12343690010CE0D39403401F52
:10527800900015E0FEA3E0FF900107E01267247498
:10528800C88E048F05FF1267148C5C8D5D800A90B0
:105298000015E0F55CA3E0F55DAE5CAF5D745E12F1
:1052A800672474058E048F05FF126714AE5AAF5B2E
:1052B800ED2FFFEC3EFE8E5C8F5DE55DF5EDE55C68
:1052C800F5EED292A203B34006E5B54420F5B590B9
:1052D80000D9E0B4025F12346390010CE0D3940764
:1052E800401BAE2CAF2D90010BE012672474C88EC2
:1052F800048F05FF1267148C5C8D5D8006852C5C1D
:10530800852D5DAE5CAF5D745E12672474058E04F6
:105318008F05FF126714AE5AAF5BED2FFFEC3EFE10
:105328008E5C8F5DE55DF5EDE55CF5EE75A700E556
:10533800B54420F5B58017123436E55DF5E9E55C2E
:10534800F5EAE55DF5EDE55CF5EED294D2928041A3
:10535800123436E55DF5E9E55CF5EAD294D292A21D
:1053680003B34008D290E5B54420F5B59000D9E0E4
:10537800B4021E123463E55DF5E9E55CF5EAE55D26
:10538800F5EDE55CF5EE75A700D290E5B54420F59E
:10539800B5D20CC20DE57090605BF82828730257EF
:0553A800F79000E0E0B9
:06605B000253A60253A946
:1053AD009060D6F8282873121DB38012121DB38099
:0E53BD000D121E3D8008121EE98003121EE92B
:0F60D6000253B40253B90253BE0253C30253C85C
:1053CB007570020257F712201512212C12244690E9
:1053DB000873E0FEA3E0FF740A12672490000AE052
:1053EB00FCA3E0FD74098F02FF1267148D078C0379
:1053FB008E048A058B06126612900877EEF0A3EFE7
:10540B00F09000C9E0B401087478BE00059F40021B
:10541B00800D7478900877F8E4F0E8A3F0801B9087
:10542B000877E0FEA3E0FF74F0BE00039F500B74FF
:10543B00F0900877F8E4F0E8A3F0E53670037536E2
:10544B0001900877E0FEA3E0FFE5362FFF50010E39
:0F545B00900877EEF0A3EFF0757003900048E033
:036061000253D116
:10546A009060E5F82828738010A230400375700A0E
:09547A008007A230400375700B9D
:0960E50002547102547302547C50
:105483000257F79006BAE0600675080112256D9081
:1054930000F9E0B401149000FAE0A852B8000495B2
:1054A300535007E55FC3956040028009741590006F
:1054B30047F00255399000AEE0D39402403F90008C
:1054C30082E02403A852B800049553500990008445
:1054D300E0D3956150028008D2027408900047F02F
:1054E300900082E0A852B80005D39553500B90006A
:1054F30084E02403C395615002C202803990008284
:10550300E02403A852B8000495535007E55FC39500
:105513006040028008D2027408900047F090008235
:10552300E0A852B80005D395535009E560240FC392
:10553300955F5002C2029000C8E07007E56AC39409
:105543001440028002D2029000BDE0B40102D202F4
:10555300A2024005757004800A757010900017E46C
:0A556300F0A3F00257F79000AEE04D
:066064000254860255699A
:10556D009060EEF8282873120E038012120E03803D
:0E557D000D120FB1800812106380031210632C
:0F60EE0002557402557902557E0255830255887A
:10558B009006BEE0600675080212256D7570050267
:10559B0057F71211A37570069006C2E060067508E6
:1055AB000312256D9006C6E0600675080412256D82
:1055BB000257F790000EE06006A204B3B3400280DE
:1055CB001D90000EE02529FFAE2850010E8E288F6E
:1055DB0029E55ED3941E500690000EE014F01213D2
:1055EB00E97570079006CAE0600675080512256D0F
:1055FB009006CEE0600675080612256D0257F790EF
:10560B0000FBE0B40203120D91121819757008908B
:10561B0006D2E0600675080712256D9006D6E0608D
:10562B000675080812256D0257F7121BD5A20CB38D
:10563B005005A20DB340028004D20CD20D75701030
:10564B009006DAE0600675080912256D9006DEE01B
:10565B00600675080A12256D0257F70257F790007E
:10566B0037E0C39446500AC296C2A07446900037E6
:10567B00F0900041E0B4011DE5362406F5369008A4
:10568B0077E0FEA3E0FF74062FFF50010E90087722
:10569B00EEF0A3EFF0900041E0B4021DE536240CD0
:1056AB00F536900877E0FEA3E0FF740C2FFF500156
:1056BB000E900877EEF0A3EFF085365B755A0090ED
:1056CB00003DE0F5731234AEE55D900037F09000CD
:1056DB0004E55AF0A3E55BF0E573900038F0C20FD8
:1056EB00900877E0F55AA3E0F55B90003DE0F57389
:1056FB001234AEE55D900035F0900000E55AF0A352
:10570B00E55BF0E573900036F0A20092109000413B
:10571B00E06002B210C20E7570030257F790003BA7
:10572B00E0C3944650139000C9E0B40102C296C284
:10573B0095C297744690003BF0900042E0B4011D77
:10574B00E5362406F536900877E0FEA3E0FF7406F5
:10575B002FFF50010E900877EEF0A3EFF090004270
:10576B00E0B4021DE536240CF536900877E0FEA375
:10577B00E0FF740C2FFF50010E900877EEF0A3EFB3
:10578B00F085365B755A0090003EE0F5731234AE2F
:10579B00E55D90003BF0900006E55AF0A3E55BF069
:1057AB00E57390003CF0C212900877E0F55AA3E045
:1057BB00F55B90003EE0F5731234AEE55D90003979
:1057CB00F0900002E55AF0A3E55BF0E57390003A28
:1057DB00F0A2009213900042E06002B213C2117566
:0C57EB00700380088006800480028000AB
:10606A0002559D0255BE02560A025635025666026E
:10607A0056690257280257EF0257F10257F302579F
:04608A00F50257F7CD
:1057F700900035E0B55E0280030258D4A20E4072D5
:10580700900000E0FEA3E0FFEF4E6021AE56AF57D9
:10581700900000E0FCA3E0FD12000374068E048FE5
:1058270005FF126714900000ECF0A3EDF09000362E
:10583700E0601A900000E0FEA3E0FFAC56AD57EF22
:105847002DFDEE3CFC900000ECF0A3EDF09000364F
:10585700E0D39401401A900000E0FEA3E0FFAC56AD
:10586700AD57EF2DFDEE3CFC900000ECF0A3EDF002
:10587700D20EAE54AF55900000E0FCA3E0FDEFC39D
:105887009DEE9C4048123FB99000C9E090608EF8A9
:105897002828738030D296802CD2968028D296D230
:1058A700A08022A2104010A223301801B34004D2D6
:1058B700A08002D296800EA223301801B34004D2F2
:0558C700968002D2A052
:0F608E0002589A02589C0258A00258A40258AA1D
:1058CC00C20E74C8900035F0A20EB3B3500790000E
:1058DC0035E0B55E028048123FB99000C9E0906097
:1058EC009DF82828738030D296802CD2968028D2AE
:1058FC0096D2A08022A2104010A223301801B340EF
:10590C0004D2A08002D296800EA223301801B3409C
:07591C0004D2968002D2A024
:0F609D000258F10258F30258F70258FB0259015A
:1059230074C8900035F0C20E900037E0B55E028077
:10593300030259CCA20F4072900004E0FEA3E0FFE3
:10594300EF4E6021AE56AF57900004E0FCA3E0FD9C
:1059530012000374068E048F05FF1267149000046F
:10596300ECF0A3EDF0900038E0601A900004E0FE44
:10597300A3E0FFAC56AD57EF2DFDEE3CFC900004C9
:10598300ECF0A3EDF0900038E0D39401401A9000BE
:1059930004E0FEA3E0FFAC56AD57EF2DFDEE3CFC5B
:1059A300900004ECF0A3EDF0D20FAE54AF5590008D
:1059B30004E0FCA3E0FDEFC39DEE9C400CC296C245
:1059C300A07446900037F0C20FA20FB3B3500790F4
:1059D3000037E0B55E02800CC296C2A07446900008
:1059E30037F0C20F900039E0B55E028003025AC45B
:1059F300A2114072900002E0FEA3E0FFEF4E60218F
:105A0300AE56AF57900002E0FCA3E0FD1200037412
:105A1300068E048F05FF126714900002ECF0A3EDCD
:105A2300F090003AE0601A900002E0FEA3E0FFACC1
:105A330056AD57EF2DFDEE3CFC900002ECF0A3EDCC
:105A4300F090003AE0D39401401A900002E0FEA3E4
:105A5300E0FFAC56AD57EF2DFDEE3CFC900002ECA1
:105A6300F0A3EDF0D211AE54AF55900002E0FCA3C9
:105A7300E0FDEFC39DEE9C4048123FB99000C9E0A2
:105A83009060ACF82828738030D296802CD2958011
:105A930028D295D2978022A2134010A22430180155
:105AA300B34004D2978002D295800EA2243018010D
:095AB300B34004D2958002D297A1
:0F60AC00025A8A025A8C025A90025A94025A9A45
:105ABC00C21174C8900039F0A211B3B35007900012
:105ACC0039E0B55E028048123FB99000C9E09060A1
:105ADC00BBF82828738030D296802CD2958028D29F
:105AEC0095D2978022A2134010A224301801B34003
:105AFC0004D2978002D295800EA224301801B340B4
:075B0C0004D2958002D2973C
:0F60BB00025AE1025AE3025AE7025AEB025AF183
:105B130074C8900039F0C21190003BE0B55E02807A
:105B230003025BC5A2124072900006E0FEA3E0FFF1
:105B3300EF4E6021AE56AF57900006E0FCA3E0FDA8
:105B430012000374068E048F05FF1267149000067B
:105B5300ECF0A3EDF090003CE0601A900006E0FE4C
:105B6300A3E0FFAC56AD57EF2DFDEE3CFC900006D5
:105B7300ECF0A3EDF090003CE0D39401401A9000C8
:105B830006E0FEA3E0FFAC56AD57EF2DFDEE3CFC67
:105B9300900006ECF0A3EDF0D212AE54AF55900096
:105BA30006E0FCA3E0FDEFC39DEE9C40159000C909
:105BB300E0B40102C296C295C297744690003BF0CE
:105BC300C212A212B3B3500790003BE0B55E02804D
:105BD300159000C9E0B40102C296C295C2977446FB
:105BE30090003BF0C2129000CBE0B40202800302AB
:105BF3005D1D90005CE0D39566506490005CE0F41A
:105C0300042566FE9000CEE08E00F5F0E884FF7E6A
:105C1300008F73EFC39410500CEF8573F0A4FDACA9
:105C2300F08D7380037573FF90005CE0D395734030
:105C33000B90005CE0C39573F57180037571009060
:105C430000E9E0D3957140069000E9E0F57190001A
:105C5300EAE0C3957150069000EAE0F57180719017
:105C6300005CE0C39566FE9000CEE08E00F5F0E8A0
:105C730084FF7E008F73EFC39410500CEF8573F095
:105C8300A4FDACF08D7380037573FF85735B755A48
:105C93000090005CE0255BFFAE5A50010E8E5A8FD8
:105CA3005B74FFBE0009D39F4005855B718003755C
:105CB30071FF9000E9E0D3957140069000E9E0F5AB
:105CC300719000EAE0C3957150069000EAE0F57127
:105CD300A204B3B3500D90005DE0FE9000D6E0D374
:105CE3009E500280147407900047F075E700E5B5F5
:105CF30054BFF5B575E710802175A71075E700E56A
:105D0300CDC395714008E5B554BFF5B58006E5B53B
:105D13004440F5B575E71075A7009000E6E0604EC6
:105D23009000F0E0A852B80004955350179000EF8C
:105D3300E0A852B8000ED3955340099000F1E0D388
:105D430095614002801575A710E5CDC394BF40044B
:105D5300C2A28002D2A275A700801375A710E5CD59
:105D6300C394404004C2A28002D2A275A70090004F
:105D7300E7E0604E9000F3E0A852B800049553505A
:105D8300179000F2E0A852B8000ED3955340099043
:105D930000F4E0D395614002801575A710E5CDC3EB
:105DA30094BF4004C2A18002D2A175A700801375DD
:105DB300A710E5CDC394404004C2A18002D2A175CF
:105DC300A700E56FC39409500AA2EDB34005C2EDE5
:105DD300122A07AE54AF557410C39F74279E400C0C
:105DE30090005BE0C3945A4003025FF5A209B340FD
:105DF30009123BF07406900047F0A20BB3500EE576
:105E030061D394334007E561C394CC4002804A9048
:105E130000FBE0B40214120D19900063E075F0501A
:105E2300A4FFAEF08E5C8F5D800F900077E075F07D
:105E330050A4FFAEF08E5C8F5DE55D455C601AA2F9
:105E430027400575FFA0D227E5B54401F5B5742DAC
:105E530090005AF0123F1BD20B90005BE0D39401E9
:105E63004007E561C3941A40028002C20B9006BA50
:105E7300E0600675080112256D9006BEE0600675A8
:105E8300080212256D9006C2E0600675080312250C
:105E93006D9006C6E0600675080412256D9006CA6B
:105EA300E0600675080512256D9006CEE060067564
:105EB300080612256D9006D2E060067508071225C4
:105EC3006D9006D6E0600675080812256D9006DA17
:105ED300E0600675080912256D9006DEE060067520
:105EE300080A12256D90005BE0C3945A5026E56FB3
:105EF300B4090990005BE004F0756F0090005BE06B
:105F0300B45A0FA227400575FFA0D227E5B5440177
:105F1300F5B5803BE56FB40903756F0075550075E2
:105F23005400758D00758B0075640090005AE0C3B2
:105F33009444500890005AE004F0800674449000A2
:105F43005AF090005AE0B44406E5B554FEF5B59016
:105F5300005BE0D394014007E56AC39441400280AB
:105F630009740E900047F0123BF0900886E060063B
:105F73009000F8E06002807A74019000BCF0900811
:105F830086E09060CAF828287380188016A2A34080
:105F93000674029000BCF0800AA2A440067402902A
:035FA30000BCF04F
:0C60CA00025F8C025F8E025F90025F9C00
:105FA6009000BCE0B40105A225B340028019D225B9
:105FB600123BF01204D574019000BCF0123310D2DB
:105FC6001F741B900047F09000BCE0B40206A225A7
:105FD600B3B340028019C225123BF01205B6740213
:105FE6009000BCF0123310D21F741B900047F002D1
:025FF60045F66E
:1060FD000000010001400160018001A001C001E02C
:10610D0002000300039603B603D603F40400050052
:10611D000512052405360548055A056C057E0590C2
:10612D0005A805C005DE0600061406280646066EFF
:10613D0006AE05CF00FF013F015F017F019F01BF4B
:10614D0001DF01FF02FF039503B503D503F303FF41
:10615D0004FF05110523053505470559056B057D1B
:10616D00058F05A705BF05CE05F1061306270645C4
:10617D00066D06AD06ED05DD0FAA0FA50F9F0F9A53
:10618D000F940F8D0F870F800F780F710F680F60B1
:10619D000F570F4E0F450F3B0F300F250F1A0F0ED8
:1061AD000F020EF50EE80EDB0ECC0EBE0EAE0E9FE0
:1061BD000E8E0E7D0E6C0E5A0E470E340E200E0CEA
:1061CD000DF70DE20DCB0DB50D9D0D850D6D0D541E
:1061DD000D3A0D200D050CE90CCE0CB10C940C767E
:1061ED000C580C3A0C1B0BFB0BDB0BBB0B9A0B79F6
:1061FD000B570B350B130AF10ACE0AAB0A870A644B
:10620D000A400A1C09F809D409B0098C0967094329
:10621D00091F08FB08D608B2088E086A084608232D
:10622D0007FF07DC07B9079607730751072F070DFF
:10623D0006EC06CA06AA068906690649062A060A52
:10624D0005EC05CD05B0059205750558053C0520F5
:10625D00050504EA04CF04B5049C048204690451C5
:10626D0004390422040B03F403DE03C803B2039DB7
:10627D00038903750361034D033B032803160304D0
:10628D0002F202E102D102C002B002A0029102822A
:10629D000273026502570249023C022F02220216C6
:1062AD00020901FD01F201E601DB01D001C601BBCE
:1062BD0001B101A7019D0194018B0182017901704A
:1062CD000168016001580150014801410139013255
:1062DD00012B0125011E01180111010B010500FF04
:1062ED0000FA0FA60FA00F990F920F8B0F840F7C42
:1062FD000F740F6B0F620F580F4E0F430F380F2C8B
:10630D000F1F0F120F050EF70EE80ED80EC80EB7A1
:10631D000EA50E930E800E6C0E580E420E2C0E1501
:10632D000DFD0DE40DCB0DB10D950D790D5D0D3FF1
:10633D000D200D010CE10CC00C9E0C7C0C590C3584
:10634D000C100BEA0BC40B9E0B760B4F0B260AFDA4
:10635D000AD40AAA0A800A550A2A09FF09D409A8EB
:10636D00097C0950092508F908CD08A10875084AC6
:10637D00081E07F307C8079D07730749072006F78F
:10638D0006CE06A6067E06570630060A05E405BFAC
:10639D00059B057705540532051004EF04CE04AEB8
:1063AD00048F047104530435041903FD03E203C77C
:1063BD0003AD0394037B0363034B0334031E0308F4
:1063CD0002F302DE02CA02B602A30291027F026D3F
:1063DD00025C024C023C022C021D020E020001F274
:1063ED0001E401D701CA01BE01B101A6019A018FD5
:1063FD000185017A01700166015D0153014A014178
:10640D00013901310129012101190112010B010489
:10641D0000FD00F700F000EA00E400DE00D900D333
:10642D0000CE00C900C400BF00BA00B500B100AD78
:10643D0000A800A400A0009C009900950091008E7A
:0C644D00008A008700840081007E007B34
:10009E0075470090087DE4F0A3F0753100753000CF
:1000AE00754D00754E00C22BD22D900886E0600271
:1000BE00D21F74FE90087FF8E4F0E8A3F074FE906F
:1000CE000883F8E4F0E8A3F074FE900881F8E4F0F9
:1000DE00E8A3F0745A9008A5F0745A9008A6F0D2CE
:1000EE002EC229C230C22FC22A22750B00750A00F9
:1000FE00AE0AAF0BAC08AD09EDC39FEC9E40167473
:10010E00FF12670475CF01780B740126F6500418A0
:10011E00E436F650DB22C2AF75D904758F0375B77E
:10012E00A575B7F190F800E4F0758F0175B7A57558
:10013E00B7F1E52790F800F075B7A575B7F190F80F
:10014E0001E4F075B7A575B7F1900899E090F80243
:10015E00F075B7A575B7F190089DE090F803F075AE
:10016E00B7A575B7F190089AE090F804F075B7A5A9
:10017E0075B7F190089BE090F805F075B7A575B7C7
:10018E00F190089CE090F806F075B7A575B7F19060
:10019E00089EE090F807F0758F0075D944D2AF2213
:1001AE00900043E0B4AB61C2AF75D90475B6227549
:1001BE00F522758F0375B7A575B7F1740090F6002B
:1001CE00F0758F01755B00755A00AE5AAF5B7413F4
:1001DE00BE00279F402475B7A575B7F1900885120C
:1001EE000048E0FC90F600120048ECF0785B7401D9
:1001FE0026F6500418E436F650D0758F0075F511BA
:10020E0075B62075D944D2AF22C2AF75F52275D915
:10021E0004755B00755A00AE5AAF5B7413BE0022B4
:10022E009F401F90F600120048E493FC9008851240
:10023E000048ECF0785B740126F6500418E436F6AC
:10024E0050D575D94475F511D2AF22900043E0B464
:10025E00AA028003020396C2AF75D90475B6227541
:10026E00F522758F0375B7A575B7F1740090EE0082
:10027E00F075B7A575B7F1740090F000F075B7A5DD
:10028E0075B7F1740090F200F075B7A575B7F174FB
:10029E000090F400F0758F01755B00755A00AE5A30
:1002AE00AF5B74FFC39F74019E402475B7A575B7ED
:1002BE00F1900073120048E0FC90EE00120048EC42
:1002CE00F0785B740126F6500418E436F650CF75BC
:1002DE005B00755A00AE5AAF5B74FFC39F74019EEC
:1002EE00402475B7A575B7F1900273120048E0FC73
:1002FE0090F000120048ECF0785B740126F6500482
:10030E0018E436F650CF755B00755A00AE5AAF5BE7
:10031E0074FFC39F74019E402475B7A575B7F19005
:10032E000473120048E0FC90F200120048ECF078E2
:10033E005B740126F6500418E436F650CF755B0058
:10034E00755A00AE5AAF5B74FFC39F74019E402472
:10035E0075B7A575B7F1900673120048E0FC90F4DE
:10036E0000120048ECF0785B740126F6500418E495
:10037E0036F650CF758F0075F51175B62075D944C8
:10038E00D2AF743A900773F022900043E0B4AA0201
:10039E0080030204D4C2AF75D90475B62275F52256
:1003AE00758F0375B7A575B7F1740090E600F075FB
:1003BE00B7A575B7F1740090E800F075B7A575B7DD
:1003CE00F1740090EA00F075B7A575B7F17400905E
:1003DE00EC00F0758F01755B00755A00AE5AAF5B7D
:1003EE0074FFC39F74019E402475B7A575B7F19035
:1003FE000073120048E0FC90E600120048ECF07822
:10040E005B740126F6500418E436F650CF755B0087
:10041E00755A00AE5AAF5B74FFC39F74019E4024A1
:10042E0075B7A575B7F1900273120048E0FC90E81D
:10043E0000120048ECF0785B740126F6500418E4C4
:10044E0036F650CF755B00755A00AE5AAF5B74FF2F
:10045E00C39F74019E402475B7A575B7F1900473C0
:10046E00120048E0FC90EA00120048ECF0785B7451
:10047E000126F6500418E436F650CF755B00755A17
:10048E0000AE5AAF5B74FFC39F74019E402475B7D4
:10049E00A575B7F1900673120048E0FC90EC0012BF
:1004AE000048ECF0785B740126F6500418E436F63A
:1004BE0050CF758F0075F51175B62075D944D2AF32
:1004CE00743A900773F022C2AF75D90475F5227590
:1004DE005B00755A00AE5AAF5B74FFC39F74019EEA
:1004EE00401F90EE00120048E493FC90007312003F
:1004FE0048ECF0785B740126F6500418E436F6509A
:10050E00D4755B00755A00AE5AAF5B74FFC39F740F
:10051E00019E401F90F000120048E493FC9002737D
:10052E00120048ECF0785B740126F6500418E4369D
:10053E00F650D4755B00755A00AE5AAF5B74FFC3AC
:10054E009F74019E401F90F200120048E493FC90AD
:10055E000473120048ECF0785B740126F650041810
:10056E00E436F650D4755B00755A00AE5AAF5B7424
:10057E00FFC39F74019E401F90F400120048E49345
:10058E00FC900673120048ECF0785B740126F6506E
:10059E000418E436F650D475F51175D944D2AF74FB
:1005AE003A900773F0C22C22C2AF75D90475F522AA
:1005BE00755B00755A00AE5AAF5B74FFC39F740132
:1005CE009E401F90E600120048E493FC90007312C8
:1005DE000048ECF0785B740126F6500418E436F609
:1005EE0050D4755B00755A00AE5AAF5B74FFC39F53
:1005FE0074019E401F90E800120048E493FC9002A4
:10060E0073120048ECF0785B740126F6500418E47F
:10061E0036F650D4755B00755A00AE5AAF5B74FF58
:10062E00C39F74019E401F90EA00120048E493FCA1
:10063E00900473120048ECF0785B740126F65004B7
:10064E0018E436F650D4755B00755A00AE5AAF5B9F
:10065E0074FFC39F74019E401F90EC00120048E48B
:10066E0093FC900673120048ECF0785B740126F64A
:10067E00500418E436F650D475F51175D944D2AF3E
:10068E00743A900773F0D22C22E54E64046006E5AE
:10069E009964FF60028031A22B4004D22B8027E5A3
:1006AE004E600874E6254E900047F0E54D600874E4
:1006BE00F0254D900047F0E54EB4010280FE754ED8
:1006CE0000754D00C22B8002C22BE54E903280F891
:1006DE00282873754E00E599B4FF03754D01E59911
:1006EE00B4FE03754D02E599B4FD03754D03E5990E
:1006FE00B4FC03754D04E599B4FA03754D05E599FF
:10070E00B4FB06754E01123BF0E599B4F906754E31
:10071E0004123BF0E599D394E54007E599C394F0B4
:10072E004002801685994F754E027E017F00E54F7F
:10073E00C394E61267248E328F3390087DE4F0A3C3
:10074E00F0E599D394C44007E599C394E64002803E
:10075E002885994F754E0374E5C3954FF533753261
:10076E0000AE32AF339060FD1266F3E493F874017D
:10077E009390087DC8F0A3C8F0D299020B77900829
:10078E0085E0700AA220B35005A221B34002804238
:10079E0090087DE0FEA3E0FF74FFBE00039F5009AA
:1007AE00EFC39446EE9406401190087DE0FEA3E060
:1007BE00FFEFD3946DEE9406401390087DE0FEA3F8
:1007CE00E0FF900073120048E599F080038599745C
:1007DE00801190087DE0FEA3E0FF900073120048A8
:1007EE00E599F090087D12673290087DE0FEA3E057
:1007FE00FFEFB40106EEB407028003020970900702
:10080E0073E0B43C028003020970A220B35005A22B
:10081E0021B340030208E7C29C900885E0900111C5
:10082E00F0900886E0900080F0900887E09000A09D
:10083E00F0900888E09000C9F0900889E09000756B
:10084E00F090088AE09000BBF090088BE09000D901
:10085E00F090088CE09000ADF090088DE09000CB09
:10086E00F090088EE09000FBF090088FE090015F12
:10087E00F0900890E0900160F0900891E090016196
:10088E00F012354990005EE09000E2F090005FE0DB
:10089E00900099F0900060E090009AF074AB900098
:1008AE0043F01201AE74AA900043F0A22CB340059F
:1008BE001203978003120259900043E4F090015FF7
:1008CE00E0700C900160E07006900161E0600280C3
:1008DE0004C2208002D220807EC29C900111E09042
:1008EE000885F0900080E0900886F09000A0E090DF
:1008FE000887F09000C9E0900888F0900075E090AD
:10090E000889F09000BBE090088AF09000D9E09042
:10091E00088BF09000ADE090088CF09000CBE0904A
:10092E00088DF09000FBE090088EF0740090088F18
:10093E00F07400900890F07400900891F074AB90F1
:10094E000043F01201AE74AA900043F01202591245
:10095E0003977599FB80FED29C754E00754D007500
:10096E0099FB020B7790087DE0FEA3E0FFEF4E703F
:10097E000685993175300090087DE0FEA3E0FF7486
:10098E00016F4E701BAC30AD31AA32AB33ED2BFB89
:10099E00EC3AFA8A068B07900073120048E599F03C
:1009AE0090087D12673290087DE0FEA3E0FF74028E
:1009BE006F4E7021AC30AD3174566D4C7006E54FF4
:1009CE0064E660028003123BF0123549854F99753B
:1009DE004E00754D00020B7790087DE0FEA3E0FF00
:1009EE00900073120048E599F090087D12673290DE
:1009FE00087DE0FEA3E0FFAC32AD338F028E038C98
:100A0E00068D079061411266F3E493F9740193FE2B
:100A1E00EAD39EEB994009854F99754E00754D00AE
:100A2E00020B7790087DE0FEA3E0FF9000731200AA
:100A3E0048E599F090087D12673290087DE0FEA39C
:100A4E00E0FFEFB40006EEB401028003020B7790D4
:100A5E000053E0D394C7400B900053E0C394C8F505
:100A6E0050801A900053E0D39463400B900053E0F3
:100A7E00C39464F5508006900053E0F550E5507530
:100A8E00F002A4FFAEF08F73EF900073126755EF74
:100A9E00FCE0FDEC900076126755EDFCE0FDEC2DD0
:100AAE00B550028003020B680FEF9000731267556A
:100ABE00E573FFE0FCEF900077126755ECFFE0FC6A
:100ACE00EFC39CB550028003020B68E5739000756E
:100ADE00126755E573FFE0FCEF900078126755EC56
:100AEE00FFE0FCEF2CB55072E5739000791267555C
:100AFE00E0C39550900899F0E57390007A1267550F
:100B0E00E0C3955090089AF0E57390007D126755FA
:100B1E00E0C3955090089BF0E57390007E126755E8
:100B2E00E0C3955090089CF0E57390007F126755D6
:100B3E00E0C3955090089DF0E573900080126755C4
:100B4E00E0C3955090089EF01201247599F97464D3
:100B5E00F5097508001200F880FE7599FF7464F5AA
:090B6E00097508001200F880FE70
:0F3280000206E102078C0209730209E6020A3115
:100B770022E54D90328FF8282873020C5C90087D8F
:100B8700E0FEA3E0FF900049120048E0F5999008C5
:100B97007D12673290087DE0FEA3E0FF74116F4E6F
:100BA7007003754D00020C5C856E99020C5C900811
:100BB7007DE0FEA3E0FF900073120048E0F599EF97
:100BC700B40107EEB40703754D0090087D12673234
:070BD700020C5C90087EE0B7
:0F328F00020B81020B84020BAF020BB5020BDAAC
:100BDE009032E3F82828738553998067855F998052
:100BEE0062856199805D8565998058856799805386
:100BFE00856899804E8569998049856A9980449067
:100C0E000018E0F599803CA22DB340077599FAC201
:100C1E002D8017A21FB3400575990F800B900047CA
:100C2E00E0F599900047E4F0C21F8017856B99801C
:100C3E0012856699800D856C9980087599FC8003E4
:030C4E00754D00E1
:1032E300020BE5020BEA020BEF020BF4020BF902ED
:1032F3000BFE020C03020C08020C0D020C15020C4F
:0D3303003A020C3F020C44020C49020C4E31
:0B0C510090087D12673280031233ED23
:03329E00020C59C6
:100C5C0022E537255BFFAE5A50010E90007312004F
:100C6C0048E0F538E537255BFFAE5A50010E0FBF53
:100C7C0000010E900073120048E0F539853F3BE50A
:100C8C0038B539058538378041E539D39538401D5D
:100C9C00E539C39538853AF0A4FFAEF0E53B8E04F8
:100CAC008F05FF126714ED2538F537801DE538C325
:100CBC009539853AF0A4FFAEF0E53B8E048F05FF25
:100CCC00126714EDF4042538F53722E539D395383D
:100CDC00401DE539C39538853AF0A4FFAEF0E53BED
:100CEC008E048F05FF126714ED2538F537801DE54E
:100CFC0038C39539853AF0A4FFAEF0E53B8E048FEE
:100D0C0005FF126714EDF4042538F53722900079AD
:100D1C00E0B40170E56775F00A84FF7E008F37E55B
:100D2C006775F00A84ADF07C008D3A753F0A755AF0
:100D3C0005755B24E537C394115005120C5D8006D4
:100D4C009005A8E0F537E537900063F0E56775F09E
:100D5C000A84FF7E008F37E56775F00A84ADF07C5E
:100D6C00008D3A753F0A755A05755B5AE537C39481
:100D7C00115005120C5D80069005DEE0F537E53765
:100D8C0090000EF022900079E0B4016AE56775F0EE
:100D9C000A84FF7E008F37E56775F00A84ADF07C1E
:100DAC00008D3A753F0A755A05755B36E537C39465
:100DBC00115005120C5D80069005BAE0F5378537A9
:100DCC004BE56775F00A84FF7E008F37E56775F099
:100DDC000A84ADF07C008D3A753F0A755A05755B37
:100DEC0048E537C394115005120C5D80069005CC74
:100DFC00E0F53785374C22E55F75F00484FF7E0003
:100E0C008F37E55F75F00484ADF07C008D3A753F4B
:100E1C0004755A01755B00E537C3943F5005120CFD
:100E2C005D80069001B2E0F5378537297528009072
:100E3C000046E075F020A4FFAEF09000C4E08E04F4
:100E4C008F05FF1267148D379000ACE0D3955F507F
:100E5C0003020F099000D0E0D3955F4010ED900194
:100E6C00B3126755E0F52B752A00020F0690009B14
:100E7C00E0D3955F4043E5379001B3126755E0F539
:100E8C0038E5379001D3126755E0F5399000D0E082
:100E9C00F404255FF53A90009BE0FE9000D0E0F45E
:100EAC00042EF53BE538B539058538378003120C2F
:100EBC00D785372B752A008041E5379001D312670F
:100ECC0055E0F538E5379001F3126755E0F53990A8
:100EDC00009BE0F404255FF53A9000ACE0FE900036
:100EEC009BE0F4042EF53BE538B5390585383780A1
:100EFC0003120CD785372B752A00020FB09000D344
:100F0C00E0D3955F5011E537900233126755E0F549
:100F1C002B752A00020FB090009CE0D3955F5043D4
:100F2C00E537900213126755E0F538E53790023338
:100F3C00126755E0F53990009CE0F404255FF53A12
:100F4C009000D3E0FE90009CE0F4042EF53BE538D5
:100F5C00B539058538378003120CD785372B752AA0
:100F6C00008041E5379001F3126755E0F538E5371D
:100F7C00900213126755E0F5399000ACE0F40425AB
:100F8C005FF53A90009CE0FE9000ACE0F4042EF586
:100F9C003BE538B539058538378003120CD78537D2
:100FAC002B752A00229000E4E0F53C753F11755A30
:100FBC0002755B00AE52AF53E53C75F00FA4FDAC6F
:100FCC00F0EDD39FEC9E4021E53C8E048F05FF1283
:100FDC006714ED75F010A4FFAEF0E55F75F01184A9
:100FEC00FD7C00ED2FF53D800EE55F75F01184FF63
:100FFC007E00EF24F0F53D853D37E55F75F01184FB
:10100C00AFF07E008F3A120C5D85373EAE52AF5377
:10101C009000E4E075F00FA4FDACF0EDD39FEC9ED6
:10102C004028755A02755B10853D37120C5D853E64
:10103C0038853739AE52AF53E53C8E048F05FF121D
:10104C00673F8D3A853C3B120CD7853729752800B4
:10105C00752B64752A00229000E4E0F53C753F1175
:10106C00755A02755B00AE52AF53E53C75F00FA498
:10107C00FDACF0EDD39FEC9E4021E53C8E048F053A
:10108C00FF126714ED75F010A4FFAEF0E56175F07A
:10109C001184FD7C00ED2FF53D800EE56175F0119E
:1010AC0084FF7E00EF24F0F53D853D37E56175F05A
:1010BC001184AFF07E008F3A120C5D85373EAE5234
:1010CC00AF539000E4E075F00FA4FDACF0EDD39FAE
:1010DC00EC9E4028755A02755B10853D37120C5DED
:1010EC00853E38853739AE52AF53E53C8E048F05BB
:1010FC00FF12673F8D3A853C3B120CD7853729751B
:10110C002800E56B6017E56BC394FE50109000D877
:10111C00E0B402099000C6E0D3940B50028017AEE5
:10112C0028AF29E56B12672474E78E048F05FF1234
:10113C0067148C288D299000AEE0B40453E55F75DC
:10114C00F00484FF7E008F37E55F75F00484ADF00A
:10115C007C008D3A753F04755A01755B00E537C309
:10116C00943F5005120C5D80069001B2E0F537AE4D
:10117C0028AF29E53712672474648E048F05FF129B
:10118C006714AE28AF29EF2DFDEE3CFC8C288D2981
:10119C00752B64752A0022900079E0B40146E5674E
:1011AC0075F00A84FF7E008F37E56775F00A84AD11
:1011BC00F07C008D3A753F0A755A05755B00E53772
:1011CC00C394115005120C5D8006900584E0F53730
:1011DC00AE2AAF2BE5372FFF50010E7464126767F0
:1011EC008E2A8F2B90007AE0B40146E56875F00AE0
:1011FC0084FF7E008F37E56875F00A84ADF07C00C3
:10120C008D3A753F0A755A05755B6CE537C39411B9
:10121C005005120C5D80069005F0E0F537AE2AAF54
:10122C002BE5372FFF50010E74641267678E2A8FDF
:10123C002B900089E0B40249E56AC3944175F0052E
:10124C0084FF7E008F37E56A75F00584ADF07C0075
:10125C008D3A753F05755A06755B00E537C39413D7
:10126C005005120C5D8006900686E0F537AE2AAF6D
:10127C002BE5372FFF50010E74641267678E2A8F8F
:10128C002B9000CBE0B402028003021342E55F75A1
:10129C00F01584FF7E008F37E55F75F01584ADF097
:1012AC007C008D3A753F15755A03755BF4E537C3B1
:1012BC00940B5005120C5D8006900472E0F537E536
:1012CC003775F0FFA4FFAEF09000CCE08E048F05D4
:1012DC00FF126714ED90005CF0E56675F078A4FFE2
:1012EC00AEF074FF8E048F05FF1267148C5A8D5B61
:1012FC0074028C068D071200398F37AC5AAD5B74B3
:10130C0004FF12673F8D3A753F04755A06755B28CA
:10131C00E537C3941D5005120C5D80069006B8E0AD
:10132C00F537AE2AAF2BE5372FFF50010E74641240
:10133C0067678E2A8F2B900078E0B4025DE56175AB
:10134C00F064A4FFAEF074081200398E5C8F5D74EB
:10135C00058E048F05FF1267148D37AE5CAF5D747C
:10136C00058E048F05FF12673F8D3A753F05755A40
:10137C0005755BDEE537C394135005120C5D8006D2
:10138C00900664E0F537AE2AAF2BE5372FFF5001FE
:10139C000E74641267678E2A8F2B9000BAE0703C33
:1013AC00900046E075F00584FF7E008F3790004674
:1013BC00E075F00584ADF07C008D3A753F05755AEB
:1013CC0005755BC0E537C3941D5005120C5D800696
:1013DC00900650E0F537E537900064F022900081DC
:1013EC00E0B401179008A0E0252BFFAE2A50010EA7
:1013FC009000D5E01267678E2A8F2B9000F9E0B42D
:10140C0001149000FAE0A852B8000495535007E577
:10141C005FC39560400280139000A3E0252BFFAEC4
:10142C002A50010E8E2A8F2B021818900081E0B4DE
:10143C000306A229B3B3400280509008A9E07010B3
:10144C009008A3E0C39405A852B800069553400237
:10145C0080109000A3E0252BFFAE2A50010E8E2A9F
:10146C008F2B9008A9E0600D9008A3E0A852B8005B
:10147C00069553400280109000A3E0252BFFAE2A66
:10148C0050010E8E2A8F2B02181890007BE0B402AC
:10149C0002800302181890007EE0602FE567D39459
:1014AC0046402890000FE0FEA3E0FF9000B9E075E5
:1014BC00F003A4FDACF0EFD39DEE9C400E9000DD4C
:1014CC00E0A852B80005D3955350030218189000A9
:1014DC00AEE0B40302800302167C85615B755A0092
:1014EC00900085E0A852B800049553500E900086E9
:1014FC00E0A85AB80005D3955B5003021679E56154
:10150C0075F002A4FFAEF074158E048F05FF126700
:10151C00148C068D07900603120048FEE0FFEE9037
:10152C00007DE0FEEF8E0088F0A4FFAEF074648EB8
:10153C00048F05FF1267148C5A8D5B900046E07582
:10154C00F018A4FFAEF09000C4E08E048F05FF12DB
:10155C0067148C068D0790061B120048AE5AAF5BC1
:10156C00E012672474648E048F05FF1267148C5A82
:10157C008D5BE565A85AB80077D3955B4072E5653D
:10158C00C3955BFFE4955AFE8E5A8F5B7428BE00A0
:10159C00039F500C755B28755A00740D900047F032
:1015AC00AE5AAF5B90007EE012672474288E048FD5
:1015BC0005FF1267148C5A8D5BAE28AF29740A8E06
:1015CC00048F05FF1267148D068C07AC5AAD5BCFE8
:1015DC00CECF120003740A8E048F05FF1267148C91
:1015EC005A8D5BAE28AF2912676F8E288F29807DAC
:1015FC00E565A85AB80004955B5072AE5AAF5BE52E
:10160C00651267678E5A8F5B7428BE00039F500C5F
:10161C00755B28755A00740D900047F0AE5AAF5B9D
:10162C0090007EE012672474288E048F05FF1267E9
:10163C00148C5A8D5BAE28AF29740A8E048F05FF6B
:10164C001267148D068C07AC5AAD5BCFCECF12004F
:10165C0003740A8E048F05FF1267148C5A8D5BAECF
:10166C0028AF29EF2DFDEE3CFC8C288D2902181893
:10167C009000C6E0855FF0A4FFAEF07405126724FD
:10168C0074071200398E5A8F5B900085E0A852B80F
:10169C00000495535012900086E075F002A4FDAC46
:1016AC00F0EFC39DEE9C4003021818E55F75F00B3C
:1016BC0084FF7E00900603120048FEE0FFEE9000CF
:1016CC007DE0FEEF8E0088F0A4FFAEF074648E0413
:1016DC008F05FF1267148C5A8D5B900046E075F0F5
:1016EC0018A4FFAEF09000C4E08E048F05FF1267C3
:1016FC00148C068D0790061B120048AE5AAF5BE0A7
:10170C0012672474648E048F05FF1267148C5A8D33
:10171C005BE565A85AB80077D3955B4072E565C365
:10172C00955BFFE4955AFE8E5A8F5B7428BE0003BE
:10173C009F500C755B28755A00740D900047F0AEE5
:10174C005AAF5B90007EE012672474288E048F05DC
:10175C00FF1267148C5A8D5BAE28AF29740A8E0465
:10176C008F05FF1267148D068C07AC5AAD5BCFCE7C
:10177C00CF120003740A8E048F05FF1267148C5A63
:10178C008D5BAE28AF2912676F8E288F29807DE57F
:10179C0065A85AB80004955B5072AE5AAF5BE5650C
:1017AC001267678E5A8F5B7428BE00039F500C75AE
:1017BC005B28755A00740D900047F0AE5AAF5B90E1
:1017CC00007EE012672474288E048F05FF126714C4
:1017DC008C5A8D5BAE28AF29740A8E048F05FF12CC
:1017EC0067148D068C07AC5AAD5BCFCECF120003BD
:1017FC00740A8E048F05FF1267148C5A8D5BAE2809
:10180C00AF29EF2DFDEE3CFC8C288D29229000D9C0
:10181C00E0B4026AE55F75F00884FF7E008F37E55F
:10182C005F75F00884ADF07C008D3A753F08755AF1
:10183C0001755BE0E537C3943F5005120C5D8006E3
:10184C00900272E0F53785372D752C00AE2CAF2D3C
:10185C00AC2AAD2B12000374648E048F05FF126743
:10186C00148C2C8D2D900076E08C068D071267243D
:10187C0074648E048F05FF1267148C2C8D2DAE288A
:10188C00AF29AC2AAD2B12000374648E048F05FFB4
:10189C001267148C288D29900076E08C068D071227
:1018AC00672474648E048F05FF1267148C288D29AD
:1018BC00A204401DAE52AF537405BE00039F5002EC
:1018CC00D204E561D394CC4008D202741190004745
:1018DC00F09000D8E0B402089000C6E0640B6002FF
:1018EC008035AE28AF29E56B12672474E78E048F20
:1018FC0005FF1267148C288D299000D9E0B40217CB
:10190C00AE2CAF2DE56B12672474E78E048F05FFA8
:10191C001267148C2C8D2D900098E05402601B9053
:10192C00008FE0A852B80012D39553400DA204B317
:10193C00B35007E561C3949A40028028AE34AF35AA
:10194C0090008DE075F002A4FDACF0EF2DFDEE3CA7
:10195C00FC74022DFD50010CE561BC0007D39D40C9
:10196C0003754301856135753400E5437003021A34
:10197C005C9000EBE0C395435003021A4E9000FBC1
:10198C00E0C394025076E56775F00A84FF7E009000
:10199C000573120048E0F55B755A00AE5AAF5B90C8
:1019AC00008EE012672474648E048F05FF12671496
:1019BC008C5C8D5D9000EBE004C395438C068D0729
:1019CC001267249000EBE08E048F05FF1267148CD5
:1019DC005C8D5DAE28AF29EF2DFDEE3CFC8C288D87
:1019EC00299000D9E0B40212AE2CAF2DAA5CAB5DED
:1019FC00EF2BFBEE3AFA8A2C8B2D80469000EBE015
:101A0C0004C39543854BF0A4FFAEF09000EBE08E41
:101A1C00048F05FF1267148C5C8D5DAE28AF29EF27
:101A2C002DFDEE3CFC8C288D299000D9E0B40212DF
:101A3C00AE2CAF2DAA5CAB5DEF2BFBEE3AFA8A2CE9
:101A4C008B2D05439000EBE0C39543500375430089
:101A5C00900098E05401601B90008CE0A852B800F4
:101A6C0012D39553400DA204B3B35007E55FC39452
:101A7C00CC4002802590008AE075F003A4FFAEF004
:101A8C00E5402FFF50010E74032FFF50010EE55F50
:101A9C00BE0007D39F4003754401855F40E5447049
:101AAC0003021B8F9000ECE0C395445003021B8192
:101ABC009000FBE0C394025076E56775F00A84FF52
:101ACC007E00900573120048E0F55B755A00AE5A23
:101ADC00AF5B90008BE012672474648E048F05FF5B
:101AEC001267148C5C8D5D9000ECE004C395448C03
:101AFC00068D071267249000ECE08E048F05FF1210
:101B0C0067148C5C8D5DAE28AF29EF2DFDEE3CFC8F
:101B1C008C288D299000D9E0B40212AE2CAF2DAADE
:101B2C005CAB5DEF2BFBEE3AFA8A2C8B2D8046904A
:101B3C0000ECE004C39544854CF0A4FFAEF090009B
:101B4C00ECE08E048F05FF1267148C5C8D5DAE2863
:101B5C00AF29EF2DFDEE3CFC8C288D299000D9E0AF
:101B6C00B40212AE2CAF2DAA5CAB5DEF2BFBEE3AA0
:101B7C00FA8A2C8B2D05449000ECE0C3954450035D
:101B8C007544009000EEE02529FFAE2850010E8E22
:101B9C00288F2990009DE0A828B8000495295009A9
:101BAC0090009DE0F5297528009000D9E0B4020D55
:101BBC0090009DE0A82CB80006952D40028009905D
:101BCC00009DE0F52D752C00229000D9E0B40102A7
:101BDC008003021CE0A204B35003021CDE9000A49C
:101BEC00E0B40168AE28AF29AC52AD5312000374B7
:101BFC003C8E048F05FF1267149000B4E0BC0010FB
:101C0C009D400D9000B6E0A828B80004952950021C
:101C1C00D203AE28AF29AC52AD53120003743C8EE4
:101C2C00048F05FF1267149000B4E0C3940ABC0043
:101C3C0015D39D40119000B6E0C39405A828B800B8
:101C4C0005D3952950028002C2038068AE28AF29C3
:101C5C00AC52AD5312000374788E048F05FF1267DB
:101C6C00149000B4E0BC00109D400D9000B6E0A8AC
:101C7C0028B8000495295004D2038038AE28AF2927
:101C8C00AC52AD5312000374788E048F05FF1267AB
:101C9C00149000B4E0C3940ABC0015D39D4011907D
:101CAC0000B6E0C39405A828B80005D395295002C6
:101CBC008002C203A203B34019AE28AF299000B52D
:101CCC00E012672474648E048F05FF1267148C284D
:101CDC008D298002C203A201B34006A202B3B35005
:101CEC0009900017E4F0A3F08024AE28AF2974000B
:101CFC00D39F74019E400C900017E528F0A3E529B2
:101D0C00F0800B74FF900017F8E4F0E8A3F090005B
:101D1C00A4E0B4011AAE28AF2974021267248E28ED
:101D2C008F29AE2CAF2D74021267248E2C8F2D9020
:101D3C0000BBE0C39403400990006FE0C3940250D1
:101D4C0035AE28AF29745E126724740A8E048F0591
:101D5C00FF1267148C288D299000D9E0B40217AEBD
:101D6C002CAF2D745E126724740A8E048F05FF123B
:101D7C0067148C2C8D2DAE28AF297402BE000AD3AB
:101D8C009F4006752902752800AE2CAF2D7402BE3B
:101D9C00000AD39F4006752D02752C00900015E5A6
:101DAC0028F0A3E529F022900046E0900373126717
:101DBC0055E0F541754264900046E0FE9000AFE0BE
:101DCC00D39E4037E55F75F00884FF7E008F37E5C2
:101DDC005F75F00884ADF07C008D3A753F08755A3C
:101DEC0003755B96E537C3941F5005120C5D800696
:101DFC00900428E0F5378537428035E55F75F008AB
:101E0C0084FF7E008F37E55F75F00884ADF07C00B1
:101E1C008D3A753F08755A03755BB6E537C3941F49
:101E2C005005120C5D8006900448E0F5378537426A
:101E3C00229000E5E0F53C753F11755A04755B0086
:101E4C00AE52AF53E53C75F00FA4FDACF0EDD39F53
:101E5C00EC9E4021E53C8E048F05FF126714ED7556
:101E6C00F010A4FFAEF0E55F75F01184FD7C00ED81
:101E7C002FF53D800EE55F75F01184FF7E00EF2499
:101E8C00F0F53D853D37E55F75F01184AFF07E00D0
:101E9C008F3A120C5D85373EAE52AF539000E5E0A1
:101EAC0075F00FA4FDACF0EDD39FEC9E4028755A55
:101EBC0004755B10853D37120C5D853E38853739CE
:101ECC00AE52AF53E53C8E048F05FF12673F8D3A3F
:101EDC00853C3B120CD7853741754264229000E556
:101EEC00E0F53C753F11755A04755B00AE52AF536B
:101EFC00E53C75F00FA4FDACF0EDD39FEC9E4021BA
:101F0C00E53C8E048F05FF126714ED75F010A4FFED
:101F1C00AEF0E56175F01184FD7C00ED2FF53D8090
:101F2C000EE56175F01184FF7E00EF24F0F53D8520
:101F3C003D37E56175F01184AFF07E008F3A120CDD
:101F4C005D85373EAE52AF539000E5E075F00FA4BF
:101F5C00FDACF0EDD39FEC9E4028755A04755B10D8
:101F6C00853D37120C5D853E38853739AE52AF53FF
:101F7C00E53C8E048F05FF12673F8D3A853C3B1282
:101F8C000CD78537417542649000E0E0B404799039
:101F9C000046E0FE9000AFE0D39E4037E55F75F061
:101FAC000884FF7E008F37E55F75F00884ADF07C08
:101FBC00008D3A753F08755A03755B96E537C394E7
:101FCC001F5005120C5D8006900428E0F53785370C
:101FDC00428035E55F75F00884FF7E008F37E55F42
:101FEC0075F00884ADF07C008D3A753F08755A0386
:101FFC00755BB6E537C3941F5005120C5D800690D7
:10200C000448E0F53785374222900079E0B4013B73
:10201C00E56775F00A84FF7E008F37E56775F00A77
:10202C0084ADF07C008D3A753F0A755A05755B12CC
:10203C00E537C394115005120C5D8006900596E0AF
:10204C00F537E5422537C39464F54290007AE0B445
:10205C00013BE56875F00A84FF7E008F37E56875F3
:10206C00F00A84ADF07C008D3A753F0A755A0575FF
:10207C005B7EE537C394115005120C5D800690060B
:10208C0002E0F537E5422537C39464F542E5412576
:10209C0042F536900081E0B4021090089FE025369E
:1020AC00FE9000D5E0F4042EF5369000D8E0D394E1
:1020BC00014040E56BC394E7501D74E7C3956BFE7C
:1020CC009008A1E08E00F5F0E884FF7E008F37E5E4
:1020DC00362537F536801CE56BC394E7FE9008A1D6
:1020EC00E08E00F5F0E884FF7E008F37E536C3956F
:1020FC0037F536A2044006E5412464F536E536D3BF
:10210C0094644009E536C39464F536800375360053
:10211C009000B1E0C3953650069000B1E0F5362240
:10212C00D201900062E0A852B800049553503E9042
:10213C000062E0A852B800049553500375360F9016
:10214C000062E004A852B80004955350037536079A
:10215C00900062E02402A852B8000495535002C2C9
:10216C0001900062E060067409900047F0C2307E76
:10217C00017F009000B7E01267249000C6E08E0447
:10218C008F05FF126714E55FBC0017D39D401390B9
:10219C0000C0E0B40204D2308002C201740A900084
:1021AC0047F0900079E0B401099000B8E0C395675E
:1021BC00400280159000CAE0A852B8000495535014
:1021CC0002C201740B900047F0900079E0B4010753
:1021DC00E567C394644002801D900110E0600D908F
:1021EC000110E0A852B80006955340028008C201C5
:1021FC00740B900047F0A20140037536009000F973
:10220C00E0B401149000FAE0A852B80004955350C1
:10221C0007E55FC39560400280209000A2E0D39454
:10222C001D400B9000A2E0C3941EF536800375365A
:10223C00007415900047F002231D900081E0B40358
:10224C0006A229B3B3400302231D9008A3E0C39454
:10225C0005A852B80004955350069008A9E06002F6
:10226C00801D9000A2E0D3941D400B9000A2E0C30F
:10227C00941EF5368003753600740C900047F09070
:10228C0008A3E0A852B80004955350069008A9E0A2
:10229C007002801D9000A2E0D3941D400B9000A210
:1022AC00E0C3941EF5368003753600740C9000471D
:1022BC00F09008A3E0A852B8000495535031900058
:1022CC00C0E0B40228D2309008A8E0FE9008A9E043
:1022DC00D39E50069008A9E0700280099008A8E4EB
:1022EC00F0C23080069008A8E004F08002C2019091
:1022FC0008A3E02405A852B800049553501390008D
:10230C00C0E0B4020A9008A9E07002D2308002C288
:10231C0001A22FB3401D9000A2E0D3941D400B905E
:10232C0000A2E0C3941EF53680037536007410903D
:10233C000047F085366C9000A2E0D3941D401890B5
:10234C000070E02536FE900046E075F01E84FC7FA0
:10235C0000EE2CF5368049900047E0640C600F903D
:10236C000047E064106007900047E0B41516900039
:10237C0070E0FE900046E075F01E84FC7F00EE2CB1
:10238C00F536801C900072E02536FE900070E02E31
:10239C00FE900046E075F01E84FC7F00EE2CF536B6
:1023AC0022900046E075F00584FF7E008F37900088
:1023BC0046E075F00584ADF07C008D3A753F0575EF
:1023CC005A03755BD69000C4E01475F00584FF7E4B
:1023DC0000E537BE00039F5005120C5D800BE537FE
:1023EC00900449126755E0F537E5379008A2F09054
:1023FC0008A2E0FE9000B3E0C39E50089000B3E04A
:10240C009008A2F022E56775F00A84FF7E00900523
:10241C0073120048E0F546E546D394644010E54657
:10242C00C3946475F00F84FF7E008F46800375465D
:10243C0000900096E02546F54622E56775F00A8483
:10244C00FF7E00900573120048E0C39469505590CC
:10245C0000E0E0C394035026900875E0FEA3E0FF73
:10246C007404120039E55F126724740F8E048F0513
:10247C00FF126714900873ECF0A3EDF08024900821
:10248C0075E0FEA3E0FF7404120039E561126724C5
:10249C00740F8E048F05FF126714900873ECF0A371
:1024AC00EDF0800F900875E0F8A3E0900873C8F089
:1024BC00A3C8F0A204401A900875E0FEA3E0FF74D4
:1024CC00031267247401120039900873EEF0A3EF25
:1024DC00F0900873E0FEA3E0FF900879E0FCA3E025
:1024EC00FDEDD39FEC9E400F900879E0F8A3E090AF
:1024FC000873C8F0A3C8F0900089E0B40262E56AE2
:10250C00C3944175F00584FF7E008F37E56A75F042
:10251C000584ADF07C008D3A753F05755A06755BE8
:10252C0014E537C394175005120C5D800690069A7B
:10253C00E0F537900873E0FEA3E0FF740A8E048F79
:10254C0005FF126714E5378C068D07126724740A91
:10255C008E048F05FF126714900873ECF0A3EDF056
:10256C0022E50875F004A4FFAEF09006B612004800
:10257C00E09032A1F8282873804C855373804790E3
:10258C0000C6E0855FF0A4FFAEF074081200398F2E
:10259C00738033856173802E85677380298568739A
:1025AC008024856973801F856A73801A856B73809C
:1025BC00158566738010856573800B856C7380063A
:0625CC00900018E0F57319
:1032A10002258402258602258B02259F0225A40280
:1032B10025A90225AE0225B30225B80225BD0225A6
:0732C100C20225C70225CC63
:1025D200E50875F004A4FFAEF09006B7120048E5D6
:1025E2000875F004A4FFAEF0E0FC9006B8120048B3
:1025F200ECFEE0FFEEC39F40030226DAE50875F029
:1026020004A4FFAEF09006B6120048E0B40441E51F
:102612000875F004A4FFAEF09006B8120048E0C3BB
:102622009573500AE508F50CD39231123E54E50831
:1026320075F004A4FFAEF09006B7120048E0D395FF
:1026420073400AE508F50CC39231123E540226D8B3
:10265200E50875F004A4FFAEF09006B7120048E05A
:10266200C395735015E50875F004A4FFAEF090060B
:10267200B8120048E0D395735002800AE508F50CC1
:10268200D39231123E54E50875F004A4FFAEF090E7
:1026920006B7120048E0D395735015E50875F004AB
:1026A200A4FFAEF09006B8120048E0C39573500A3A
:1026B200E508F50CC39231123E549006BEE0B40117
:1026C200099000D2E0D395615002800A7402F50CA1
:1026D200C39231123E54806AE50875F004A4FFAE3D
:1026E200F09006B7120048E0D395734015E50875DF
:1026F200F004A4FFAEF09006B8120048E0C3957350
:102702004002800AE508F50CC39231123E54E508F6
:1027120075F004A4FFAEF09006B7120048E0C3952E
:10272200734015E50875F004A4FFAEF09006B812E8
:102732000048E0D39573400AE508F50CD3923112B4
:102742003E5422AE2EAF2F74C9BE000CD39F400858
:10275200782E12677702285F752F01752E00AE5210
:10276200AF53E546BE000DD39F40099000A8E0D3C9
:10277200954740028023754700E546C39553F5739C
:102782009000ABE0D395454008E5452573F54580BB
:10279200069000ABE0F54580020547900084E0D347
:1027A2009561401CE55FC395604015AE52AF53E59D
:1027B20046BE00039F50099000A9E0D3954840020D
:1027C200806E9008A4E0A852B80004955350037597
:1027D2004A009008A4E0A852B8000BD395534006D3
:1027E200E5539008A4F0E54A7041E553C39546F5D8
:1027F20073E573D3940540037573059000AAE0C393
:1028020095455007E573C3954540028009E545C3E8
:102812009573F54580069000AAE0F5459000AAE080
:10282200D3954540069000AAE0F545754800800220
:102832000548E54A7016900084E0C39561500DE5A5
:10284200462405A852B8000695534002800F900016
:1028520097E0F545754A0174789008A4F022AE2EEF
:10286200AF2F74E9D39F74039E4008782E126777C6
:10287200022A06752F01752E00754532A22A402ABA
:10288200754519900097E075F002A4FFAEF0E54798
:10289200BE0006D39F4002D22A0547754A037478C8
:1028A2009008A4F07549000229EDAE52AF53E546F7
:1028B2006F4E70030229EDE546BE000DD39F40091D
:1028C2009000A8E0D395474002800F754700E54A83
:1028D200C394035003754519800DE546C39553F51E
:1028E20073E5472573F547900084E0D39561400E68
:1028F2009008A4E0A852B80007D395534002800C78
:102902000549900097E0B54903754A00E54AB403CA
:1029120006A204B3B34002800A0549E549B43C0368
:10292200754A02E54AB402299008A4E0A852B80008
:102932000ED395534009E5539008A4F075490090D1
:102942000084E0C39561500975490074789008A429
:10295200F0E54A705A900084E0D39561401CE55F2F
:10296200C395604015AE52AF53E546BE00039F507B
:10297200099000A9E0D39548400280087548007587
:10298200454B8028E553C39546F573E573D394050B
:102992004003757305900084E0D395614008E548D3
:1029A2002573F5488006E5482406F548754900E593
:1029B2004A7016900084E0C39561500DE5462405E7
:1029C200A852B80006955340028003754A01E54AB1
:1029D200B401187545190549900097E0B549067587
:1029E2004A0275490074789008A4F0A202B3400329
:1029F200754532E54575F00AA4FFAEF090087BEE0E
:102A0200F0A3EFF022E56F9032C8F8282873900007
:102A12007CE07003022C449000B2E0B40102800317
:102A2200022B4F900044E0655E6009E55345526019
:102A320003022B4C7E017F00E5BE126724E5BD2F09
:102A4200FF50010E8E5A8F5B741012672490006142
:102A5200E08E048F05FF12671490087FECF0A3ED5F
:102A6200F0E56B600FE56BC394FE50089000D8E070
:102A72006402600280649000C6E0B40B1F90087F7D
:102A8200E0FEA3E0FF74E7126724E56B8E048F0576
:102A9200FF12671490087FECF0A3EDF09000C6E0FF
:102AA200D3940B40089000AEE064046002802B9047
:102AB200087FE0FEA3E0FF900883E0FCA3E0FDEFC7
:102AC200D39DEE9C400D12676F90087FEEF0A3EF4E
:102AD200F0800790087FE4F0A3F090007CE0B4025D
:102AE20027900881E0FEA3E0FF90087FE0FCA3E0CE
:102AF200FDEF2DFDEE3CFC74018C068D07120039B2
:102B020090087FEEF0A3EFF090087FE0FEA3E0FFD5
:102B1200900881E0FCA3E0FDEDD39FEC9E4004D23F
:102B22002E8002B22E90087FE0F8A3E0900881C8C0
:102B3200F0A3C8F09000AEE064016006A22EB3B329
:102B420040028006900880E0F55F022C42D22E7E81
:102B5200017F00E5BE126724E5BD2FFF50010E8EF6
:102B62005A8F5B7410126724900061E08E048F0507
:102B7200FF12671490087FECF0A3EDF0E56B600F95
:102B8200E56BC394FE50089000D8E06402600280B6
:102B9200649000C6E0B40B1F90087FE0FEA3E0FF44
:102BA20074E7126724E56B8E048F05FF1267149099
:102BB200087FECF0A3EDF09000C6E0D3940B400840
:102BC2009000AEE064046002802B90087FE0FEA3D8
:102BD200E0FF900883E0FCA3E0FDEFD39DEE9C4074
:102BE2000D12676F90087FEEF0A3EFF08007900858
:102BF2007FE4F0A3F090007CE0B40227900881E02B
:102C0200FEA3E0FF90087FE0FCA3E0FDEF2DFDEEC8
:102C12003CFC74018C068D0712003990087FEEF09F
:102C2200A3EFF090087FE0F8A3E0900881C8F0A33A
:102C3200C8F09000AEE064016006900880E0F55FA5
:102C42008003755F00900078E07006756F01022ABC
:102C52000775BB1802327B900078E07003022DCA20
:102C62007E017F00E5BE126724E5BD2FFF50010EF5
:102C72008E5A8F5B9000BEE0B4010F7E0F7FFFACD7
:102C82005AAD5B12676F8E5A8F5B9000E3E0B4021D
:102C920045AE5AAF5B900021E0FCA3E0FDEDD39F6F
:102CA200EC9E400A900021E55AF0A3E55BF0AE5A93
:102CB200AF5B900023E0FCA3E0FDEFD39DEE9C40D0
:102CC2000A900023E55AF0A3E55BF0AE5AAF5B74BD
:102CD200041200398F619000E3E0704CAE5AAF5B92
:102CE200900021E0FCA3E0FDEFD39DEE9C40091291
:102CF200676F8E5A8F5B8006755B00755A00AE5AFD
:102D0200AF5B741012672490005EE08E048F05FFA3
:102D12001267148C5A8D5B74FFBC0009D39D400569
:102D2200855B6180037561FE9000AEE0B4010280B4
:102D320003022DC8A204B3B3500E900082E0A85241
:102D4200B80005D39553500280719000BFE08561B1
:102D5200F0A4FFAEF074648E048F05FF1267148C2A
:102D62005A8D5BE56B6016E56BC394FE500F9000C5
:102D7200D8E0B402089000C6E0640B60028017AE8F
:102D82005AAF5B74E7126724E56B8E048F05FF125E
:102D920067148C5A8D5BAE5AAF5B90087FE0FCA340
:102DA200E0FDEDD39FEC9E4005855B5F800BA22E7C
:102DB200B34006900880E0F55F800BA22EB3400678
:102DC200900880E0F55F800375610090007BE07001
:102DD20006756F02022A0775BB1902327B90007BCF
:102DE200E07003022E7FE55ED395514003022E7DF3
:102DF20090001FE0FEA3E0FFE56512676790001FE9
:102E0200EEF0A3EFF07E017F00E5BE126724E5BD80
:102E12002FFF50010E8E5A8F5B9000E8E070137402
:102E22000A12672474518E048F05FF1267148D6590
:102E32008019AE5AAF5B740A1267248F048E057E26
:102E4200017F95CDCCCD1266128F65E565D3946472
:102E5200400375656490001FE0FEA3E0FFE5652F67
:102E6200FF50010E90001FEEF0A3EFF090007FE004
:102E7200048E048F05FF1267148D65800375653219
:102E82009000CBE07006756F03022A0775BB130230
:102E9200327B9000CBE0604A7E017F00E5BE126784
:102EA20024E5BD2FFF50010E8E5A8F5B7404120071
:102EB200398F669000CDE08566F0A4FDACF07464B5
:102EC200FF1267148D669000CCE08566F0A4FFAE19
:102ED200F074FF8E048F05FF126714ED90005DF011
:102EE2008003756600900079E07006756F04022A0F
:102EF2000775BB1702327B900079E0B401028003B0
:102F0200022F8D7E017F00E5BE126724E5BD2FFFF3
:102F120050010E8E5A8F5B9008A5E060199008A5AB
:102F2200E01490618512008CE493FC740193FDED32
:102F3200C39FEC9E400280069008A5E014F0900822
:102F4200A5E0C394B3501DAE5AAF5B9008A5E00450
:102F520090618512008CE493FC740193FDEFC39D94
:102F6200EE9C400280069008A5E004F09008A5E0DF
:102F7200FE90009FE08E0088F0A4FFAEF074648E95
:102F8200048F05FF1267148D678003756700900038
:102F92007AE07006756F05022A0775BB1602327B4E
:102FA20090007AE0B4010280030230367E017F0095
:102FB200E5BE126724E5BD2FFF50010E8E5A8F5BCE
:102FC2009008A6E060199008A6E0149062EF120043
:102FD2008CE493FC740193FDEDC39FEC9E40028050
:102FE200069008A6E014F09008A6E0C394B3501D22
:102FF200AE5AAF5B9008A6E0049062EF12008CE438
:1030020093FC740193FDEFC39DEE9C4002800690F9
:1030120008A6E004F09008A6E0FE9000A5E08E006D
:1030220088F0A4FFAEF074648E048F05FF1267145B
:103032008D68800375680075BB1F02327B7E017F3D
:1030420000E5BE126724E5BD2FFF50010E8E5A8F98
:103052005B740912672474E68E048F05FF126714ED
:103062008D6A900081E07006756F07022A0775BBB2
:103072001502327B900081E070030231C77E017F2E
:1030820000E5BE126724E5BD2FFF50010E8E5A8F58
:103092005B74041200398F69900081E0B4011590CD
:1030A20000D5E08569F0A4FFAEF07407120039EF95
:1030B2009008A0F0900081E0B402159000D5E08560
:1030C20069F0A4FFAEF07407120039EF90089FF088
:1030D200900081E0B4030280030231AA9000C2E0B2
:1030E2007052E569C39419500FD2299000A1E09063
:1030F20008A3F09008A7E4F0E569D394644004A221
:10310200294002802D9008A7E004F09008A7E0FE75
:10311200900114E0B5060B9008A3E004F09008A714
:10312200E4F09008A3E064966006900114E0700257
:10313200C22980639000A1E070349000D5E08569D7
:10314200F0A4FFAEF074FF8E048F05FF126714ED3A
:103152009008A3F0AE52AF53741EBE0006D39F4038
:1031620002D229E561D394E54002C2298029E569AA
:10317200C3940A500DAE52AF53741EBE0004D39FC7
:1031820050028002D229E561D394E54002C229901F
:1031920000A1E09008A3F09008A3E0C394055006B4
:1031A20074059008A3F0C22F900081E0B40414E5E6
:1031B20069C394195002D22FE569D394324002C2F6
:1031C2002FC22980037569009000D8E07006756FE0
:1031D20008022A0775BB1402327B9000D8E0700304
:1031E20002326A7E017F00E5BE126724E5BD2FFF31
:1031F20050010E8E5A8F5B9000FDE07025EFD39444
:1032020021EE940E4005756BFF8015AE5AAF5B74CC
:103212001012672474E38E048F05FF1267148D6BFE
:103222008027AE5AAF5BEFD39449EE940640057502
:103232006BFF8015AE5AAF5B741012672474658EF3
:10324200048F05FF1267148D6BE56B75F00BA4FFFD
:10325200AEF09000C6E08E048F05FF12671490084E
:1032620083ECF0A3EDF08003756B0090007CE060CE
:093272000575BB1A800375BB1839
:1032C800022A10022C59022DDF022E94022EF90236
:0B32D8002FA202303F0230760231DCF2
:05327B00056FD2EC22FA
:096755002582F582500205832221
:0F008C0025E050020583258250020583F582226C
:1066F300EF2F500205832582F582E5833E2EF58335
:016703002273
:10676700CFC39FFF50011E22C3EF9DFFEE9CFE2269
:086777000806B6000218062214
:0D673200A3E004F0700612674BE004F022B3
:0E003900048007C3CE13CECF13CFD5E0F6223E
:10661200BC000FBE0008ED8FF084FFADF022E4FE57
:10662200FF22BE000DEF60FE54F0606F20E7030210
:1066320066C8EAC0E0EBC0E078017A0075F001EECE
:1066420020E710EF25E0FFEE33FE0AC5F023C5F088
:1066520030E7F0EA5407F9096A7A007B0060010822
:10666200C3EC9E40167004ED9F4010ED9FFDEC9E22
:10667200FCE5F0CA4ACA03F5F08005E5F003F5F03F
:10668200C3EE13FEEF13FFD9D77908CACBCAD8D00D
:10669200EAFEEBFFD0E0FBD0E0FA22EC8FF084FCC4
:1066A200ED54F045F0C48FF084FEEDC454F045F093
:1066B200C48FF084FDEEC4FE54F02DFFEE540F3C67
:1066C200FEADF07C0022790078008FF0EC7E08208D
:1066D200E70DC3CD33CD33C933C9C833C8DEF08427
:1066E20049F9E5F08FF0BE00E6FD7C00E9FFE8FE27
:0166F2002285
:0E672400F88FF0A4FFE5F0CE88F0A42EFE2240
:10000300EF8DF0A4F9A8F0EF8CF0A428F8EE8DF0B2
:06001300A428FEE9FF2213
:10670400600D782B02670E007830D8FED5E0F822B1
:10671400EEC0E07E00126612EFFDEEFCD0E0FE2239
:0C673F00EEC0E07E00126612D0E0FE22E8
:03001B0002001EC2
:0300530002005652
:03009B00020071EF
:0300000002675E36
:09675E0075817575D0000240F050
:0B004800E5822FF582E5833EF5832260
:0A674B000582D58202158315822213
:10001E00C0E0C0F0C083C082C0D075D000123FEEE9
:0B002E00D0D0D082D083D0F0D0E032E0
:10005600C0E0C0F0C083C082C0D075D000123FF1AE
:10006600D0D0D082D083D0F0D0E032C0E0C0F0C093
:1000760083C082C0D075D0001240B2D0D0D082D01A
:0600860083D0F0D0E0324F
:00000001FF
